:100000000C94D6000C9493220C94BE220C94BF2323
:100010000C9400000C9400000C9400000C94000060
:100020000C9400000C9400000C9400000C94000050
:100030000C9400000C94A40F0C9400000C9400008D
:100040000C9400000C9400000C9400000C94000030
:100050000C940000010000004843000048430000E9
:100060004843020000000000000000000000000003
:10007000000048E1FA3ECDCC4C3D0AD7A33B6F12BD
:10008000033A17B75138ACC5A73600256642256636
:100090004100314235303041000025302E30667449
:1000A0000025302E30667500300025302E30667603
:1000B0000025302E3066770025302E3066780025FA
:1000C000302E3066790025302E31667A0025302EAC
:1000D0003166210025302E3066400025302E3066F6
:1000E000230025302E3066240025302E3066260071
:1000F00025302E30665E0025302E306666002530B5
:100100002E3066670025302E3066680025302E3090
:1001100066690025302E30666A0025302E30666B09
:100120000025302E30666C0025302E30666D00259F
:10013000302E30666E0025302E30666F0025302E52
:100140003066700025302E3066710025302E306606
:10015000720025302E3066A30025302E3266A500B1
:1001600025302E3266830025302E3266E1002530A0
:100170002E3066ED0025302E3066B10025302E3051
:1001800066F30025302E3066BA0000000200F90246
:1001900054000400FB0256000400FF025A00040051
:1001A00003035E000200090362000000F894EE27DA
:1001B000ECBBF1E0FBBFEBBFE5BFF8E1F1BDE1BD9A
:1001C0008DE0A2E0BB27ED938A95E9F780E098E007
:1001D000A0E6ED930197E9F7ECE8F1E085919591C0
:1001E000009761F0A591B59105901590BF01F001C0
:1001F00005900D920197E1F7FB01F0CFEFE5EDBF20
:10020000E8E0EEBFC0E6D2E00C94F025A49A089591
:10021000A498AC9A0895AC9A0895AC980895AD9AB4
:100220000895AD980895A59AAD980E940801089583
:100230000E94002E0E94062E0E940D0183E48A95E2
:10024000F1F70E9411010E94062E0E940B0183E427
:100250008A95F1F70E94110108950A930E94002ED9
:1002600000E00A3038F40E94122E83E48A95F1F7F8
:100270000F5FF7CF0E941801099108951A930A930E
:1002800010E00E94080100E8E0E0E01758F40E9446
:100290000F0183E48A95F1F79C99102B0E941101BC
:1002A0000695F2CF0E9406010E940D010E94122EB7
:1002B0000E940801E12F0991199108951A930A9358
:1002C00010E00E94060100E8E0E0E017A0F4EA81F7
:1002D000E02319F00E940B0102C00E940D010E9450
:1002E0000F0183E48A95F1F783E48A95F1F70E9480
:1002F00011010695E9CF0E9408010E940F0183E4D5
:100300008A95F1F7E0E09C99E1E01E2F0E9411012F
:10031000E12F19810881239608950E94D53B0FEFA4
:100320001FEF0E941801EC81EA930E945E0130E009
:10033000343130F49C9B04C00E94192E3F5FF8CFEB
:100340009C9913C00E943E01F0E00E2F1F2F102F2A
:1003500000270E943E01A02FB12FF0E0EA0FFB1F03
:100360000E2F1F2F0E943E012E2FE02FF12F0E94F3
:10037000DC3B259608950E94C837E0936103ECECBE
:100380000E941F2EE4E40E941F2EC39A0895C39872
:100390000E94C837E0936103E5E50E941F2E08958F
:1003A000C1989798949A959A0895E1E0F0E0E093C7
:1003B0001D03F0931E03A5E2B0E00E94253AE894E5
:1003C00025F8E0E0E093CD02E093CE020E94252ED6
:1003D0000895E0915F03F0916003309711F00C9461
:1003E0006A02EC2DFD2DEB5BFF4FFF93EF930E9414
:1003F000312EE081AF91BF910E942D3AEC2DFD2D61
:10040000E755FF4FFF93EF930E94312EE181AF91AB
:10041000BF910E942D3AEC2DFD2DE35FFE4FFF931F
:10042000EF930E94312EE281AF91BF910E942D3A4D
:10043000EC2DFD2DEF58FE4FFF93EF930E94312ED0
:10044000E381AF91BF910E942D3AEC2DFD2DEB522F
:10045000FE4FFF93EF930E94312EE481AF91BF9145
:100460000E942D3AEC2DFD2DE75CFD4FFF93EF939D
:100470000E94312EE581AF91BF910E942D3AEC2D63
:10048000FD2DE356FD4FFF93EF930E94312EE68141
:10049000AF91BF910E942D3AEC2DFD2DEF5FFC4FE7
:1004A000FF93EF930E94312EE781AF91BF910E949D
:1004B0002D3AC0925B03D0925C03A3E4B0E00E94AB
:1004C0000A3A31960E94253A3197EC2DFD2D31964E
:1004D000CE2EDF2E0895ECE50E943C2E0895E0E537
:1004E0000E943C2E0895E091BD02F091BE0232962A
:1004F000E093BD02F093BE02A091BD02B091BE0296
:10050000EFEFF0E0EA17FB079CF4E091BF02F091F7
:10051000C0023196E093BF02F093C002E091BD02A9
:10052000F091BE02E050F140E093BD02F093BE02B4
:100530000895E0911503F0911603309711F4C19AD4
:10054000979A0E94402E0E94D0010895E091600287
:10055000A091A802EA17C1F5E091A902EF93E091FA
:100560006102AF91EA1781F5E091AA02EF93E09161
:100570006202AF91EA1741F5E091AB02EF93E0918F
:100580006302AF91EA1701F5E091AC02EF93E091BD
:100590006402AF91EA17C1F4E091AD02EF93E091EC
:1005A0006502AF91EA1781F4E091AE02EF93E0911A
:1005B0006602AF91EA1741F4E091AF02EF93E09148
:1005C0006702AF91EA1709F006C0E1E0F0E0E093BE
:1005D0005903F0935A030895C19A0E94462EC19878
:1005E00008950E94312EE081E0934C030E94312E49
:1005F000E181E0934D030E94312EE281E0934E03AE
:100600000E94312EE381E0934F030E94312EE4815A
:10061000E09350030E94312EE581E09351030E9444
:10062000312EE681E09352030E94312EE781E09360
:1006300053030895E0904C03E0914D03E09345038C
:10064000E0914E03E0934603E0914F03E0934703AC
:10065000E0915003E0934803E0915103E093490394
:10066000E0915203E0934A03E0915303E0934B037C
:100670000895E0E0E0935D03E0935E03E0E0E09343
:100680005F03E0936003A0915D03B0915E03AC153E
:10069000BD0514F00C94C503AB5BBF4F0E940E3A2E
:1006A000A0914C03EA1711F00C94AC03A0915D03E8
:1006B000B0915E03A755BF4F0E940E3AA0914D0323
:1006C000EA1711F00C94AC03A0915D03B0915E03A6
:1006D000A35FBE4F0E940E3AA0914E03EA17E1F5C8
:1006E000A0915D03B0915E03AF58BE4F0E940E3AD9
:1006F000A0914F03EA1781F5A0915D03B0915E03CD
:10070000AB52BE4F0E940E3AA0915003EA1721F55A
:10071000A0915D03B0915E03A75CBD4F0E940E3AAD
:10072000A0915103EA17C1F4A0915D03B0915E035B
:10073000A356BD4F0E940E3AA0915203EA1761F4EE
:10074000A0915D03B0915E03AF5FBC4F0E940E3A73
:10075000A0915303EA1709F00EC0E1E0F0E0E09346
:100760005F03F0936003E0915D03F0915E03E0931B
:100770005B03F0935C03E0915D03F0915E033196BF
:10078000E0935D03F0935E037ECF0895AF9A88EC0B
:1007900090E00197F1F70E944C2E88EC90E00197D1
:1007A000F1F70E944F2E0E944F2E0E944F2E0E9462
:1007B000522E0E94552E0E94552E0E94522E88ECD9
:1007C00090E00197F1F7AF980E94EC0208950E9423
:1007D000D53BAF9A8BE18A95F1F70E944F2E0E948C
:1007E0004F2E0E94582E8BE18A95F1F70E944F2ED2
:1007F000EA930E94B3371E2F8BE18A95F1F7AF98E9
:100800008BE18A95F1F7003011F0002331F0E2E03E
:10081000F0E0E0934303F0934403EEE0E01730F49C
:10082000E3E0F0E0E0934303F0934403EDE1E017ED
:1008300030F4E4E0F0E0E0934303F0934403ECE2AF
:10084000E01730F4E1E0F0E0E0934303F093440379
:10085000AF9A0E945D2EA0914303B0914403A13052
:10086000E0E0BE0711F40E944F2EA0914303B09127
:100870004403A230E0E0BE0711F40E94632EA09171
:100880004303B0914403A330E0E0BE0711F40E949B
:10089000662EA0914303B0914403A430E0E0BE076C
:1008A00011F40E94692E8BE18A95F1F7AF988BE1E4
:1008B0008A95F1F7AF9A0E946C2E8BE18A95F1F739
:1008C000AF988BE18A95F1F7AF9A0E94732E8BE176
:1008D0008A95F1F7AF988BE18A95F1F7AF9A0E946C
:1008E0007A2E8BE18A95F1F7AF98E12FF0E02E2F69
:1008F0003F2F2F5F3F4FA0914303B0914403A1309E
:10090000E0E0BE0711F42F5F3F4FEBE3F0E0E217AA
:10091000F30764F420E030E0A0914303B091440376
:10092000A130E0E0BE0711F421E030E0E22FF32F28
:10093000EA930E94BF371E2F8BE18A95F1F7AF9A99
:100940008BE18A95F1F7EBE8EA930E94F92DA091EB
:100950004303B0914403A130E0E0BE0711F40E94CC
:100960004F2EA0914303B0914403A230E0E0BE07B4
:1009700011F40E94632EA0914303B0914403A3306D
:10098000E0E0BE0711F40E94662EA0914303B091EF
:100990004403A430E0E0BE0711F40E94692E8BE10D
:1009A0008A95F1F7AF988BE18A95F1F7AF9A8BE1D1
:1009B0008A95F1F7ECE8EA930E94F92D1A930E94C8
:1009C000F92D8BE18A95F1F7AF988BE18A95F1F7D4
:1009D000AF9A8BE18A95F1F7EDE80E94812E8BE1C9
:1009E0008A95F1F7AF988BE18A95F1F7AF9A8BE191
:1009F0008A95F1F7EEE80E94812E8BE18A95F1F756
:100A0000AF980E94DC3B2496089524970A93AF9AEE
:100A10008BE18A95F1F70E944F2E0E944F2E0E9483
:100A2000582E0E94842E0E94582EE02FF0E0E09372
:100A3000EB02F093EC020E94842E0E2F0A930E9488
:100A4000B3370E2F0E94922EE093E902F093EA0250
:100A50008BE18A95F1F7AF988BE18A95F1F7AF9A20
:100A60000E94522E0E944F2E0E94582E0E94922EBB
:100A7000E093ED02F093EE020E944F2E0E94582E5A
:100A80000E94922EE093EF02F093F0020E944F2E0C
:100A90000E94582E0E94922EE093F102F093F202EF
:100AA0008BE18A95F1F7AF98088125960895DE9835
:100AB0008BE08A95F1F7DF988BE08A95F1F7E88172
:100AC000F981EBBB8BE08A95F1F7DF9A8BE18A9590
:100AD000F1F7E0ECEBBB0E949F2E22960895289739
:100AE0000E94D33BA0911103B0911203A430E0E027
:100AF000BE0709F4AA98E1E0F0E0E715F80529F04F
:100B0000E3E0F0E0E715F80511F4A89A01C0A89811
:100B1000A091F902B091FA02A130E0E0BE0779F4A9
:100B2000A0913B03B0913C03A130E0E0BE0739F453
:100B3000A0911303B09114030E94BB3B09F00BC0BA
:100B4000C49A0E94A52E0E94B12E0E94B72E969A9A
:100B5000C098AB9A7FC2C4989698A0911103B091A7
:100B60001203A130E0E0BE07E9F4E091B902F09190
:100B7000BA026091BB027091BC020E94BD2E11F4BA
:100B80000E94C92EAE85BF85888999890E94C33B82
:100B90001CF40E94E62E02C00E94F12EEE87FF8711
:100BA000688B798BA0911103B0911203A230E0E021
:100BB000BE07C9F4A9E0B0E00E94053A0E94BD2E2C
:100BC00011F40E94C92EAE85BF85888999890E943B
:100BD000C33B1CF40E94E62E02C00E94F12EEE8759
:100BE000FF87688B798BA0911103B0911203A3301A
:100BF000E0E0BE07C1F4A3E1B0E00E94053A0E9424
:100C0000983AEE87FF87688B798BAE85BF85888998
:100C10009989E0E0F0E060E271E40E94563BEE87E3
:100C2000FF87688B798BA0911103B0911203A430D8
:100C3000E0E0BE0729F4E0E0EE87EF87E88BE98B80
:100C4000E0911103F0911203309791F5E2E0F0E0AA
:100C5000E715F805E1F40E94FE2E0E9410390E946B
:100C6000983AEE83FF8368877987AE81BF81888554
:100C70009985E0E0F0E068EC72E40E94563BEE8378
:100C8000FF8368877987EE87FF87688B798BE3E03E
:100C9000F0E0E715F80561F4E0910303F091040337
:100CA0006091050370910603EE87FF87688B798B4F
:100CB000AE85BF8588899989E0E0F0E064E573E45A
:100CC0000E94973B10F00C941408C09AA09139032D
:100CD000B0913A03A130E0E0BE0789F4E09111033E
:100CE000F0911203309759F400240714080429F0F6
:100CF000E1E0F0E0E715F80511F40E94C92EAE8599
:100D0000BF8588899989E0E0F0E060E271E40E94A3
:100D1000243B0E94653A0E2F1F2F0E940D2F09F0D1
:100D200010F40C949606C0980E94182FE2E0F0E0B0
:100D3000E715F80509F4C09AA0911103B0911203C8
:100D4000A430E0E0BE0791F4E0E0EE87EF87E88BA7
:100D5000E98B4EE050E0ECE0F0E0EC87FD87EAE064
:100D6000F0E0FA93EA930E9457056BC000501040E0
:100D7000F4F4E02FF12F0E94DD380E2F1F2F0436E0
:100D8000E0E01E071CF4C09AAA9A04C00E94182F23
:100D9000C098AA9A2FE030E0A02FB12F0E94212FF7
:100DA0000E94282F0E942F2FEC87FD8746C00E94AB
:100DB0000D2F09F010F40C94DF06C09801C0C09A02
:100DC000AA98A02FB12FE4E6F0E00E9476392E2FEA
:100DD0003F2F0E94352FDF010E94212F0E94352FC7
:100DE000FF93EF930E94282FAF91BF91AE1BBF0BD3
:100DF000AC87BD87E2E0F0E0E715F805F1F4E0919B
:100E00001103F09112033097C1F4A091EB02B0915D
:100E1000EC02EAE0F0E00E947639EC87FD87AC85D1
:100E2000BD85EAE0F0E00E944639A091EB02B09166
:100E3000EC02AE1BBF0BAA87BB873A932A930E9492
:100E40005705E42FF52F7096FA93EA930E94570501
:100E5000EC85FD85B096FA93EA930E945705A09120
:100E60001103B0911203A430E0E0BE07A1F4AB98E7
:100E7000A0911303B0911403A130E0E0BE0719F470
:100E8000E0E3F0E002C0E1E3F0E0FA93EA930E94CD
:100E90005705C098C8C034FE08C0EDE3F0E0FA93EF
:100EA000EA930E945705AB98BEC0072C082859F555
:100EB000A091F902B091FA02A530E0E0BE0711F46A
:100EC00035FC01C009C0EBE3F0E0FA93EA930E941D
:100ED0005705E89435F816C0AB98E0913903F091C6
:100EE0003A03309719F40E94B72E0CC00E943C2F91
:100EF00034FE08C0C09A0E940D2F09F010F40C9423
:100F00008207C09890C0AB98E1E0F0E0E715F805E3
:100F100011F00C94CA07E0911103F091120330977D
:100F200011F5A091F902B091FA02A530E0E0BE07F8
:100F300019F40E94422F16C0E0913903F0913A0350
:100F4000309719F40E94B72E0DC00E943C2F34FE3A
:100F500009C00E940D2F09F010F40C94B107C0983D
:100F600001C0C09A16C0E0913903F0913A0330975E
:100F700019F40E94B72E0DC00E943C2F34FE09C008
:100F80000E940D2F09F010F40C94C807C09801C0FE
:100F9000C09A49C0E2E0F0E0E715F80529F5E091D4
:100FA0001103F0911203309741F4EA85FB85F09626
:100FB000FA93EA930E94570516C0E0913903F09125
:100FC0003A03309719F40E94B72E0DC00E943C2FAF
:100FD00034FE09C00E940D2F09F010F40C94F207A2
:100FE000C09801C0C09A1FC0E3E0F0E0E715F80523
:100FF00021F40E94422FAB9A16C0E0913903F09180
:101000003A03309719F40E94B72E0DC00E943C2F6E
:1010100034FE09C00E940D2F09F010F40C94120840
:10102000C09801C0C09A16C0ECE0F0E0FA93EA93D1
:101030000E945705EAE1F0E0FA93EA930E9457050F
:101040000E94B12EE1E3F0E0FA93EA930E94570583
:10105000969AC098A0911103B0911203A130E0E0DC
:10106000BE0739F4A0913703B09138030E94BB3B0F
:1010700081F0A0911103B0911203A230E0E0BE070D
:1010800039F4A0913503B09136030E94BB3B09F0BF
:101090000CC0C098AA9A0E94A52EEFE2F0E0FA9345
:1010A000EA930E9457050E943C2FA0911103B09132
:1010B00012030E94BB3B54F4A898A5E6B3E00E943B
:1010C0000A3AE130A0E0FA0709F4A89A0E94DA3B54
:1010D000629608950E94482F31F10E94C70155245D
:1010E000E8E05E1648F4E52DF0E0E855FD4FE081BC
:1010F0000E941F2E5394F4CFEEEB0E941F2E00E0AF
:1011000010E00930E0E01E0764F40E94592FFF93BD
:10111000EF930E940938AF91BF91EC930F5F1F4F7F
:10112000F0CF0E94602F0E94822F09F010F40C94DF
:101130009B080E94972FE889F9896A897B890E9418
:10114000653AE093C902F093CA020E94A82F3BC0FF
:101150000E94482F61F10E94C7015524E8E05E1605
:1011600038F40E94312EDF010E94B72F5394F6CF3E
:10117000EEEB0E941F2E00E010E00930E0E01E07B9
:1011800064F40E94592FFF93EF930E940938AF91A6
:10119000BF91EC930F5F1F4FF0CF0E94602F0E9412
:1011A000822F09F010F40C94D7080E94972FE88939
:1011B000F9896A897B890E94653AE093CB02F093B2
:1011C000CC020E94A82F19810881649608950E947C
:1011D000402EAF9A88EC90E00197F1F70E94BD2F66
:1011E0000E944F2E8BE18A95F1F7AF9A0E945D2EF7
:1011F0008BE18A95F1F70E944C2E8BE18A95F1F7ED
:101200000E944C2E8BE18A95F1F70E944C2E8BE1C7
:101210008A95F1F70E944C2E8BE18A95F1F7AF98F1
:101220008BE18A95F1F7AF9A8BE18A95F1F70E94ED
:10123000BD2FE7E0EA930E94F92D8BE18A95F1F743
:10124000AF9AAF9A0E945D2E0E944C2E8BE18A9538
:10125000F1F7AF988BE18A95F1F7AF9A0E946C2E67
:101260008BE18A95F1F7AF988BE18A95F1F7AF9A08
:101270000E94732E8BE18A95F1F7AF988BE18A95E6
:10128000F1F7AF9A0E947A2E8BE18A95F1F7AF9829
:10129000089564970E94D43BE4E6EB1549F50E945B
:1012A000C02FF4F4EAE8F0E0BE2E0E94D32FE091C4
:1012B000E102F091E2026091E3027091E4020E9487
:1012C000983AE987FA876B877C87EBE8F0E00E9421
:1012D000EC2F88E00E94DA2D2A96E89433F808C0B3
:1012E000E2E9F0E0FA93EA9380E00E94DA2D229698
:1012F000E3E6EB1511F00C944A0AE9E9F0E0BE2EA2
:10130000E091BD02F091BE020E941039E093E50227
:10131000F093E6026093E7027093E802E091BF0267
:10132000F091C002FE2FE0E0A091E502B091E6024C
:101330008091E7029091E8020E9410390E94D8380B
:10134000E093E502F093E6026093E7027093E8020F
:101350000E94983AED8BFE8B6F8B788FA091E10203
:10136000B091E2028091E3029091E402E8E00E94F1
:10137000F638EB8BFC8BE8E00E94EA38E98BFA8BBD
:101380000E940239E98BFA8BE091E102F091E202CE
:101390006091E3027091E4020E94983A0E94FF2F4C
:1013A0000E94243BED83FE836F837887E091E50202
:1013B000F091E6026091E7027091E802AD81BE8192
:1013C0008F8198850E94983A0E94563B0E94FF2F79
:1013D0000E94CF3AED83FE836F8378870E94F339B2
:1013E0000E946F050E94C02F14F00C94420A0E94C4
:1013F0006F0283E08A95F1F7AE980E940C300B895A
:101400000A930E94F92D09890E9412301E2F0E9412
:101410004F2E2E2F83E08A95F1F7AE9A83E08A95BE
:10142000F1F70E946B02E091E102F091E20260911B
:10143000E3027091E402EE5FFF4F6F4F7F4FE09346
:10144000E102F093E2026093E3027093E4020E94EF
:101450001530E32FF42F0E9410390E94983AE09340
:101460000D03F0930E0360930F03709310030E941B
:10147000D32FEBE8F0E00E94EC2F88E00E94DA2DF9
:101480002A9608C0E2E9F0E0FA93EA9380E00E942D
:10149000DA2D22960E94DB3B699608950E94A808E7
:1014A000E093FF02F0930003609301037093020343
:1014B0000E9424300895AE980E944530AE9A83E091
:1014C0008A95F1F7AE980E944F30E091BF020E94DA
:1014D0005530E091BD020E94553008952C9782E06E
:1014E000A0E0B0E0E4E6F0E00E94E13B0E94D33BE4
:1014F00001E010E021E030E042E050E0E0913B0309
:10150000F0913C03309711F00C94E20EF894EEEF5A
:10151000FFE7EC87FD870E940239E88BF98BEC85A9
:10152000FD85FE2FE0E0EE87FF870E940239EE87FF
:10153000FF878BE18A95F1F7E3E50E943C2E40910D
:101540003F0350914003A0910903B0910A03A130D9
:10155000E0E0BE0739F4E0913F03F091400332969A
:101560004E2F5F2F25FEE9C242E050E0A091F70226
:10157000B091F802A03AE0E0BE07C1F4A091E90200
:10158000B091EA02ECE3F0E00E944639A091EB0250
:10159000B091EC02EA0FFB1FE093C902F093CA027C
:1015A000ECEBFFE7E093CB02F093CC02A091F702C3
:1015B000B091F802AA3AE0E0BE0711F00C94720C68
:1015C000A091F102B091F2020E94BB3B14F00C9486
:1015D000720CAA30E0E0BE07DCF40E945930FF93A1
:1015E000EF930E946230AF91BF91EA0FFB1FA09171
:1015F000F102B091F202EA0FFB1FE093C902F093EF
:10160000CA02E6ECFFE7E093CB02F093CC026AC19A
:10161000A091F102B091F202A431E0E0BE0704F51E
:101620000E945930FF93EF930E946230AF91BF91B7
:10163000EA0FFB1FFF93EF93E091F102F091F202AA
:101640003A97AF91BF91EA0FFB1FE093C902F09365
:10165000CA02E7ECFFE7E093CB02F093CC0242C171
:10166000A091F102B091F202AE31E0E0BE0704F5C4
:101670000E945930FF93EF930E946230AF91BF9167
:10168000EA0FFB1FFF93EF93E091F102F091F2025A
:101690007497AF91BF91EA0FFB1FE093C902F093DB
:1016A000CA02E8ECFFE7E093CB02F093CC021AC148
:1016B000A091F102B091F202A832E0E0BE0704F579
:1016C0000E945930FF93EF930E946230AF91BF9117
:1016D000EA0FFB1FFF93EF93E091F102F091F2020A
:1016E0007E97AF91BF91EA0FFB1FE093C902F09381
:1016F000CA02E9ECFFE7E093CB02F093CC02F2C020
:10170000A091F102B091F202A233E0E0BE0704F52D
:101710000E945930FF93EF930E946230AF91BF91C6
:10172000EA0FFB1FFF93EF93E091F102F091F202B9
:10173000B897AF91BF91EA0FFB1FE093C902F093F6
:10174000CA02EAECFFE7E093CB02F093CC02CAC0F6
:10175000A091F102B091F202AC33E0E0BE0704F5D3
:101760000E945930FF93EF930E946230AF91BF9176
:10177000EA0FFB1FFF93EF93E091F102F091F20269
:10178000F297AF91BF91EA0FFB1FE093C902F0936C
:10179000CA02EBECFFE7E093CB02F093CC02A2C0CD
:1017A000A091F102B091F202A634E0E0BE0704F588
:1017B0000E945930FF93EF930E946230AF91BF9126
:1017C000EA0FFB1FFF93EF93E091F102F091F20219
:1017D000FC97AF91BF91EA0FFB1FE093C902F09312
:1017E000CA02ECECFFE7E093CB02F093CC027AC0A4
:1017F000A091F102B091F202A035E0E0BE070CF535
:101800000E945930FF93EF930E946230AF91BF91D5
:10181000EA0FFB1FFF93EF93E091F102F091F202C8
:10182000E654F040AF91BF91EA0FFB1FE093C9026D
:10183000F093CA02EDECFFE7E093CB02F093CC0209
:1018400051C0A091F102B091F202AA35E0E0BE07CA
:101850000CF50E945930FF93EF930E946230AF91D4
:10186000BF91EA0FFB1FFF93EF93E091F102F0911C
:10187000F202E055F040AF91BF91EA0FFB1FE093F9
:10188000C902F093CA02EEECFFE7E093CB02F093BB
:10189000CC0228C0A091F102B091F202A436E0E09F
:1018A000BE0704F50E945930FF93EF930E94623007
:1018B000AF91BF91EA0FFB1FFF93EF93E091F1020D
:1018C000F091F202EA55F040AF91BF91EA0FFB1F91
:1018D000E093C902F093CA02EFECFFE7E093CB027A
:1018E000F093CC02A091F702B091F802A43BE0E0A3
:1018F000BE0761F4A9E0B0E00E94053A0E946B3097
:10190000E0EDFFE7E093CB02F093CC02A091F70269
:10191000B091F802AE3BE0E0BE0761F4ADE0B0E0AC
:101920000E94053A0E946B30EAEDFFE7E093CB029C
:10193000F093CC02A091F702B091F802A83CE0E04D
:10194000BE0771F4A3E1B0E00E94053AE093C9023A
:10195000F093CA02E4EEFFE7E093CB02F093CC02EF
:10196000A091F702B091F802A23DE0E0BE0761F558
:10197000A0910903B0910A03A130E0E0BE0749F449
:10198000E0913F03F09140033296E093C902F09357
:10199000CA02A0910903B0910A03A230E0E0BE0799
:1019A00069F4E0913F03F0914003309709F002C0E1
:1019B000E1E0F0E0E093C902F093CA02EEEEFFE747
:1019C000E093CB02F093CC02A091F702B091F80221
:1019D000A33DE0E0BE0771F4A0915B03B0915C030E
:1019E000AB5BBF4F0E947830EFEEFFE7E093CB0296
:1019F000F093CC02A091F702B091F802A43DE0E090
:101A0000BE0771F4A0915B03B0915C03A755BF4F73
:101A10000E947830E0EFFFE7E093CB02F093CC0236
:101A2000A091F702B091F802A53DE0E0BE0771F485
:101A3000A0915B03B0915C03A35FBE4F0E9478301E
:101A4000E1EFFFE7E093CB02F093CC02A091F70225
:101A5000B091F802A63DE0E0BE0771F4A0915B03EF
:101A6000B0915C03AF58BE4F0E947830E2EFFFE7C1
:101A7000E093CB02F093CC02A091F702B091F80270
:101A8000A73DE0E0BE0771F4A0915B03B0915C0359
:101A9000AB52BE4F0E947830E3EFFFE7E093CB02FA
:101AA000F093CC02A091F702B091F802A83DE0E0DB
:101AB000BE0771F4A0915B03B0915C03A75CBD4FBE
:101AC0000E947830E4EFFFE7E093CB02F093CC0282
:101AD000A091F702B091F802A93DE0E0BE0771F4D1
:101AE000A0915B03B0915C03A356BD4F0E94783078
:101AF000E5EFFFE7E093CB02F093CC02A091F70271
:101B0000B091F802AA3DE0E0BE0771F4A0915B033A
:101B1000B0915C03AF5FBC4F0E947830E6EFFFE707
:101B2000E093CB02F093CC020E9480300E949B3065
:101B300001E010E021E030E084C0A091DF02B0912C
:101B4000E0020E94BB3B4CF4E091D502F091D6023A
:101B50006091D7027091D80202C0E0ECF8E0E09307
:101B6000C902F093CA02A091C902B091CA021097AB
:101B700014F40E94B6300E948030E091DF02F091B0
:101B8000E002A091D902B091DA028091DB0290913B
:101B9000DC020E9410390E94A139E093C902F0933F
:101BA000CA02E091D902F091DA026091DB027091F1
:101BB000DC02E093C902F093CA02A091C902B0917D
:101BC000CA02109714F40E94B630E091C902F09155
:101BD000CA020E9402390E2F1F2FE091C902F09114
:101BE000CA02FE2FE0E02E2F3F2F232F332727FDA1
:101BF0003095A091DD02B091DE020E94BB3B4CF417
:101C0000E091D102F091D2026091D3027091D4029E
:101C100002C0E0ECF8E0E093CB02F093CC02A0919C
:101C2000CB02B091CC02109744F4E0E6F9E0EA1B55
:101C3000FB0BE093CB02F093CC020E949B300E94FE
:101C4000C330E091BD02F091BE02E887F987E091D0
:101C5000BF02F091C002EA87FB8725FE03C00E9405
:101C6000D7301DC0A0910903B0910A03A130E0E074
:101C7000BE0729F4E2E0F0E0E417F50774F0A09164
:101C80000903B0910A03A230E0E0BE0729F4E1E0C5
:101C9000F0E0E417F5070CF002C00E94D730AE81E7
:101CA000BF81A130E0E0BE0789F40E945B0AE091A9
:101CB000C1020E945530E091C3020E94553088EC69
:101CC00090E00197F1F7AE9A0E94462EA091090389
:101CD000B0910A03A130E0E0BE07A9F425FC13C0CF
:101CE0000E9473020E945B0A009358030E94DD3039
:101CF000209358030E94DD3088EC90E00197F1F7C3
:101D0000AE9A0E94462E0E9473020E945B0AE889E6
:101D10000E945530EE850E94553088EC90E0019786
:101D2000F1F7AE9A0E94462EAE9888EC90E00197AB
:101D3000F1F7E6E00E94E130AE9A88EC90E001977E
:101D4000F1F7AE9888EC90E00197F1F7E2E0EA93C2
:101D50000E94F92DEA850E945530E8850E94553091
:101D6000AE81BF81A130E0E0BE0739F4E091C50249
:101D70000E945530E091C70206C0E091C1020E9466
:101D80005530E091C302E09358030E94DD3088ECA7
:101D900090E00197F1F7AE9A0E94462E0E946B02E6
:101DA000A091BF02B091C002AF37E0E0BE0749F496
:101DB0000E94E83034F4E1E0F0E0E0933B03F0937C
:101DC0003C0378940E94DA3B62960895689425F863
:101DD0000E94462E0E94F1300E94FA300E94033188
:101DE0000E94462E0E940B310E94462E0E94133103
:101DF0000E94462E0895689425F80E94F1300E94B2
:101E0000FA300895689425F8E0EAF0E0E093F702EC
:101E1000F093F802689431F8EAEAF0E0E093F70210
:101E2000F093F802689432F8089528970E94D33B03
:101E3000EEEFFFE7EE83FF830E9402394E2F5F2F04
:101E4000EE81FF81FE2FE0E0E887F9870E940239EA
:101E5000E887F987E0E0E093E102E093E202E093B3
:101E6000E302E093E402E0E0E093CD02E093CE02EF
:101E7000E0E0E093BD02E093BE02E0E0E093BF0249
:101E8000E093C0020E94462E0E946F0283E08A9572
:101E9000F1F7E0E0EA87EB87EC87ED8700E010E000
:101EA00020E030E0AA85BB858C859D85AD3FEFE7BE
:101EB000BE07E0E08E07E0E09E07ACF5AE980E941A
:101EC0004530AE9A83E08A95F1F7AE980E944F3084
:101ED000209358030E94DD30009358030E94DD30A8
:101EE000409358030E94DD30E8850E94553083E01E
:101EF0008A95F1F7AE9A0E5F1F4FEA85FB856C85D8
:101F00007D85EE5FFF4F6F4F7F4FEA87FB876C87C2
:101F10007D87EFEFF0E0E017F10724F42F5F3F4FEC
:101F200000501140BFCF83E08A95F1F70E946B0209
:101F30000E94EC020E94192E0E94EC020C940000F8
:101F40000E94DA3B2E96089568970A93BCB0689475
:101F500020F8E89423F8E0E0E0930703E093080317
:101F6000E4E2EB1511F00C94B90F0C94003C0C94C6
:101F70001B1DE8E7EB1531F4F8940E94150F7894D7
:101F80000C941B1DE6E2EB1511F5F894E0E0E093EC
:101F9000E102E093E202E093E302E093E402E0E096
:101FA000E093CD02E093CE020E94E60E0E941B3128
:101FB0000E94462EE89425F80E94C330E89434F835
:101FC0000E9429310E94E70378940C941B1DE3E6DC
:101FD000EB15E9F4E0E0E093CD02E093CE026894E3
:101FE00034F8E0E0E0931103E093120377248824AF
:101FF000E89423F8E89433F8E0E0E0934103E093B9
:1020000042030E9437310E94D0010C941B1DE4E66C
:10201000EB15A1F4E0E0E093CD02E093CE02E8946A
:1020200023F8E0E0E0931103E0931203772488247F
:10203000689433F80E9437310C941B1DE7E5EB15CB
:1020400011F00C94D9120E943F31EAE9F0E00E94AD
:102050004C3184E00E945531E1EAF0E00E944C31BD
:1020600084E00E94643140F4E8EAF0E0FA93EA93F5
:1020700080E00E94DA2D2296EAEAF0E00E944C31DC
:1020800084E00E94DA2D26960E947D310E948A31DA
:1020900040F4E8EAF0E0FA93EA9380E00E94DA2D57
:1020A0002296E1EBF0E00E944C3184E00E949531F1
:1020B00040F4E8EAF0E0FA93EA9380E00E94DA2D37
:1020C0002296E8EBF0E00E944C3184E00E94DA2D89
:1020D0002696E0911303F09114030E9410390E9498
:1020E000983AED8BFE8B6F8B788FEFEBF0E00E94D0
:1020F0004C3184E00E94DA2D2696A0913903B091EC
:102100003A03A130E0E0BE0731F5A9E0B0E00E945B
:10211000053AE98BFA8B6B8B7C8BE6ECF0E0FA935B
:10212000EA93AB89BC898D899E890E94A43184E0A1
:102130000E94DA2D2696EDECF0E0FA93EA93A09156
:10214000B902B091BA028091BB029091BC020E9488
:10215000A43184E025C0A9E0B0E00E94053AE98BF3
:10216000FA8B6B8B7C8BE6ECF0E0FA93EA93EB89CD
:10217000FC896D897E890E94F33984E00E94DA2D02
:102180002696EDECF0E0FA93EA93E091B902F09133
:10219000BA026091BB027091BC020E94F33984E0E4
:1021A0000E94DA2D2696E0913903F0913A030E94BD
:1021B00010390E94983AED8BFE8B6F8B788FE4ED8F
:1021C000F0E00E944C3184E00E94BB31EBEDF0E086
:1021D0000E944C3184E00E94DA2D2696A3E1B0E003
:1021E0000E94053A0E94983AED8BFE8B6F8B788F98
:1021F000E2EEF0E00E944C3184E00E94DA2D269657
:102200000E94CA31E9EEF0E00E944C3184E00E9465
:10221000D731E0EFF0E00E944C3184E00E94DA2DEB
:1022200026960E94E431E7EFF0E00E944C3184E012
:102230000E94DA2D26960E94F131EEEFF0E00E9426
:102240004C3184E00E94DA2D26960E94FE310E94D5
:102250008A3140F4E8EAF0E0FA93EA9380E00E94E1
:10226000DA2D2296E5E0F1E00E944C3184E00E94F4
:10227000DA2D26960E940B320E948A3140F4E8EA59
:10228000F0E0FA93EA9380E00E94DA2D2296ECE0E7
:10229000F1E00E944C3184E00E94DA2D26960E94E3
:1022A00018320E948A3140F4E8EAF0E0FA93EA93A7
:1022B00080E00E94DA2D2296E3E1F1E00E944C31A9
:1022C00084E00E94DA2D26960E942532EAE1F1E0B0
:1022D0000E944C3184E00E94DA2D26960E94323210
:1022E000E1E2F1E00E944C3184E00E94DA2D269672
:1022F0000E943F320E948A3140F4E8EAF0E0FA930B
:10230000EA9380E00E94DA2D2296E8E2F1E00E9452
:102310004C3184E00E94DA2D26960E944C320E94B5
:102320008A3140F4E8EAF0E0FA93EA9380E00E9410
:10233000DA2D2296EFE2F1E00E944C3184E00E9417
:10234000DA2D26960E9459320E948A3140F4E8EA3A
:10235000F0E0FA93EA9380E00E94DA2D2296E6E319
:10236000F1E00E944C3184E00E94DA2D2696E09143
:102370001903F0911A030E9410390E94983AED8BCC
:10238000FE8B6F8B788FEDE3F1E00E944C3184E09F
:102390000E94DA2D2696A0911B03B0911C03A13058
:1023A000E0E0BE0711F00C942D12A0911903B0913A
:1023B0001A03A130E0E0BE0711F00C9424120E9431
:1023C0006632FF93EF930E946F32AF91BF910E94EC
:1023D0007832ED87FE876F87788B0E948332E9879A
:1023E000FA876B877C870E949432FF93EF930E9459
:1023F0009D32AF91BF910E94A632ED83FE836F8321
:1024000078870E94B132E983FA836B837C830E94D0
:10241000C2321CF40E94CD3216C00E94C23289F42E
:10242000E985FA856B857C85A981BA818B819C8140
:102430000E94C93B1CF40E94CD3202C00E94DA32D5
:1024400002C00E94DA3208C0E0E0F0E060E87FE31A
:10245000ED8BFE8B6F8B788F05C0E0E0ED8BEE8B04
:10246000EF8BE88FE4E4F1E00E944C3184E00E94BD
:10247000DA2D2696E0913303F09134030E9410394F
:102480000E94983AED8BFE8B6F8B788FEBE4F1E036
:102490000E944C3184E00E94DA2D2696E62DFF271B
:1024A000662777270E94983AED8BFE8B6F8B788F8B
:1024B000E2E5F1E00E944C3184E00E94DA2D26969C
:1024C000E9E5F1E0FA93EA93E091FB02F091FC0276
:1024D0006091FD027091FE020E94F33984E00E9437
:1024E000DA2D2696E0E6F1E0FA93EA93E091FF0216
:1024F000F091000360910103709102030E94F3398F
:1025000084E00E94DA2D2696E7E6F1E0FA93EA935A
:10251000E0910303F09104036091050370910603B9
:102520000E94F33984E00E94DA2D2696ADE3B0E0F4
:102530000E940A3A0E9410390E94983AED8BFE8B55
:102540006F8B788FEEE6F1E00E944C3184E00E94C0
:10255000DA2D2696E0916603F09167030E94103908
:102560000E94983AED8BFE8B6F8B788FE5E7F1E058
:102570000E944C3184E00E94DA2D2696AFE3B0E051
:102580000E940A3A0E9410390E94983AED8BFE8B05
:102590006F8B788FECE7F1E00E944C3184E00E9471
:1025A000DA2D2696E0E0E0930703E09308030C940D
:1025B0001B1DE1E4EB1579F4E0E0F0E0A7E1B0E009
:1025C0000E94253AE0E0E0933903E0933A030E9449
:1025D00029310C941B1DE2E4EB1571F4E1E0F0E00D
:1025E000A7E1B0E00E94253AE0933903F0933A0363
:1025F0000E9429310C941B1DE3E4EB15D1F5949A4C
:10260000959A0E94E83209F010F40C941013A9E096
:10261000B0E00E94053AADECBCEC8CEC9DE308C048
:10262000A9E0B0E00E94053AA0E0B0E080E89FE3B6
:102630000E94D63AA9E0B0E00E941A3A0E94F53210
:1026400009F010F40C942C13E0E0F0E06AEF72E46F
:10265000A9E0B0E00E941A3A0E94023394980E94C6
:102660000D3325F80E941B3326F80E94EC020C94CF
:102670001B1DE4E4EB1569F5949A959A0E94E832E3
:1026800009F010F40C9447130E94233302C00E94F7
:102690002E330E94F8390E94CF3AA9E0B0E00E94A0
:1026A0001A3A0E94393340F4E0E0F0E068E472EC5A
:1026B000A9E0B0E00E941A3A0E94023394980E9466
:1026C0000D3325F80E941B3326F80E94EC020C946F
:1026D0001B1DE5E4EB1511F00C94B713949A959A31
:1026E0000E94463309F010F40C948313A091B902B0
:1026F000B091BA028091BB029091BC02EDECFCEC6F
:102700006CEC7DE30CC0A091B902B091BA0280914B
:10271000BB029091BC02E0E0F0E060E87FE30E9441
:10272000F8390E94CF3AE093B902F093BA0260936D
:10273000BB027093BC020E94553360F4E0E0F0E00D
:1027400068E472ECE093B902F093BA026093BB02C2
:102750007093BC020E94643395980E940D3325F853
:102760000E947D3327F80E94EC020C941B1DE6E4C6
:10277000EB1511F00C940614949A959A0E94463326
:1027800009F010F40C94D113E091B902F091BA025F
:102790006091BB027091BC02ADECBCEC8CEC9DE393
:1027A0000CC0E091B902F091BA026091BB02709145
:1027B000BC02A0E0B0E080E89FE30E94D63AE0933C
:1027C000B902F093BA026093BB027093BC020E94FC
:1027D000853309F010F40C94F913E0E0F0E068ECB4
:1027E00072E4E093B902F093BA026093BB02709373
:1027F000BC020E94643395980E940D3325F80E9414
:102800007D3327F80E94EC020C941B1DE7E4EB15C6
:1028100009F50E949433A3E1B0E00E94053AE1304B
:10282000A0E0FA07A0E06A07A0E07A074CF4E1E034
:10283000F0E060E070E0A3E1B0E00E941A3A08C066
:102840000E940D3325F80E94A13330F80E94EC025B
:102850000C941B1DE8E4EB1561F40E94A9330E945F
:102860000D3325F80E94A13330F80E94EC020C943D
:102870001B1DEBE2EB1559F5949A959AA9E0B0E08F
:102880000E94053AA0E0B0E080E89FE30E94D63ABB
:10289000A9E0B0E00E941A3A0E94F53209F010F463
:1028A0000C945A14E0E0F0E06AEF72E4A9E0B0E0C2
:1028B0000E941A3A0E94023394980E940D3325F820
:1028C0000E941B3326F80E94EC020C941B1DEDE7BE
:1028D000EB1521F5949A959A0E942E330E94F839AF
:1028E0000E94CF3AA9E0B0E00E941A3A0E94393320
:1028F00040F4E0E0F0E068E472ECA9E0B0E00E94AF
:102900001A3A0E94023394980E940D3325F80E94CF
:102910001B3326F80E94EC020C941B1DEBE5EB1513
:10292000B1F5949A959AA091B902B091BA028091AA
:10293000BB029091BC02E0E0F0E060E87FE30E941F
:10294000F8390E94CF3AE093B902F093BA0260934B
:10295000BB027093BC020E94553360F4E0E0F0E0EB
:1029600068E472ECE093B902F093BA026093BB02A0
:102970007093BC020E94643395980E940D3325F831
:102980000E947D3327F80E94EC020C941B1DEDE59C
:10299000EB15B9F5949A959AE091B902F091BA02C3
:1029A0006091BB027091BC02A0E0B0E080E89FE3C0
:1029B0000E94D63AE093B902F093BA026093BB0248
:1029C0007093BC020E94853309F010F40C94F41447
:1029D000E0E0F0E068EC72E4E093B902F093BA0250
:1029E0006093BB027093BC020E94643395980E946E
:1029F0000D3325F80E947D3327F80E94EC020C94D9
:102A00001B1DEAE3EB1551F5A3E1B0E00E94053A86
:102A1000EA50F04060407040A3E1B0E00E941A3AF2
:102A2000A3E1B0E00E94053AE130A0E0FA07A0E09F
:102A30006A07A0E07A0744F4E1E0F0E060E070E0CB
:102A4000A3E1B0E00E941A3A0E940D3325F80E94DB
:102A5000A13330F80E94EC020C941B1DEBE3EB1544
:102A6000B1F4A3E1B0E00E94053AE65FFF4F6F4F7B
:102A70007F4FA3E1B0E00E941A3A0E940D3325F87F
:102A80000E94A13330F80E94EC020C941B1DE9E473
:102A9000EB15E1F4A1E1B0E00E940A3A31970E94FF
:102AA000253A3196A1E1B0E00E940A3AE130A0E077
:102AB000FA0734F4E1E0F0E0A1E1B0E00E94253A49
:102AC0000E94CA310E9429310C941B1DEAE4EB15C7
:102AD00071F4A1E1B0E00E940A3A31960E94253AD1
:102AE00031970E94CA310E9429310C941B1DEBE4DE
:102AF000EB1529F5E091E902F091EA023196E093B5
:102B0000E902F093EA02A091E902B091EA02E7E15A
:102B1000F0E0EA17FB072CF4E0E0E093E902E09331
:102B2000EA020E94020F0E947D31AF9A0E94B633E2
:102B30000E94BC33AF980E94EC020C941B1DECE485
:102B4000EB1511F5E091E902F091EA023197E0937B
:102B5000E902F093EA02A091E902B091EA0210972B
:102B600034F4E7E1F0E0E093E902F093EA020E9436
:102B7000020F0E947D31AF9A0E94B6330E94BC338F
:102B8000AF980E94EC0257C7EDE4EB1511F5E09108
:102B9000EB02F091EC023196E093EB02F093EC0241
:102BA000A091EB02B091EC02EBE3F0E0EA17FB0737
:102BB0002CF4E0E0E093EB02E093EC020E94CC33D3
:102BC000AF9A0E94DB330E94E133AF980E94EC027F
:102BD00032C7EEE4EB1501F5E091EB02F091EC0267
:102BE0003197E093EB02F093EC02A091EB02B091ED
:102BF000EC02109734F4EBE3F0E0E093EB02F09397
:102C0000EC020E94CC33AF9A0E94DB330E94E13386
:102C1000AF980E94EC020FC7EFE4EB1511F00C9493
:102C2000E216E091ED02F091EE0231960E94F1334E
:102C3000E1F0A091EF02B091F002A330E0E0BE0716
:102C4000A1F0A530E0E0BE0781F0A730E0E0BE07CC
:102C500061F0A830E0E0BE0741F0AA30E0E0BE0736
:102C600021F0AC30E0E0BE0779F4A091ED02B09124
:102C7000EE02EFE1F0E0EA17FB0734F4E1E0F0E008
:102C8000E093ED02F093EE02A091EF02B091F0021A
:102C9000A430E0E0BE0761F0A630E0E0BE0741F0FE
:102CA000A930E0E0BE0721F0AB30E0E0BE0779F4E8
:102CB000A091ED02B091EE02EEE1F0E0EA17FB0721
:102CC00034F4E1E0F0E0E093ED02F093EE02A09145
:102CD000EF02B091F002A230E0E0BE0711F00C94D8
:102CE000D216A091F102B091F202A430E0E0BE074A
:102CF00011F40C94B316A830E0E0BE0711F40C9464
:102D0000B316AC30E0E0BE0711F40C94B316A0315A
:102D1000E0E0BE0711F40C94B316A431E0E0BE0766
:102D200011F40C94B316A831E0E0BE07E1F0AC3129
:102D3000E0E0BE07C1F0A032E0E0BE07A1F0A4329F
:102D4000E0E0BE0781F0A832E0E0BE0761F0AC32FF
:102D5000E0E0BE0741F0A033E0E0BE0721F0A4337D
:102D6000E0E0BE0781F4A091ED02B091EE02EDE14A
:102D7000F0E0EA17FB0734F4E1E0F0E0E093ED0265
:102D8000F093EE020FC0A091ED02B091EE02ECE1E3
:102D9000F0E0EA17FB0734F4E1E0F0E0E093ED0245
:102DA000F093EE020E94020F0E943F31AF9A0E9400
:102DB000FD330E940334AF988BE18A95F1F70E94AE
:102DC000EC0239C6E0E5EB1511F00C94B7178BE176
:102DD0008A95F1F7E091ED02F091EE0231970E94B1
:102DE000F133E1F0A091EF02B091F002A330E0E006
:102DF000BE07A1F0A530E0E0BE0781F0A730E0E01B
:102E0000BE0761F0A830E0E0BE0741F0AA30E0E084
:102E1000BE0721F0AC30E0E0BE0771F4A091ED02F6
:102E2000B091EE02A130E0E0BE0734F4EFE1F0E053
:102E3000E093ED02F093EE02A091EF02B091F00268
:102E4000A430E0E0BE0761F0A630E0E0BE0741F04C
:102E5000A930E0E0BE0721F0AB30E0E0BE0771F43E
:102E6000A091ED02B091EE02A130E0E0BE0734F493
:102E7000EEE1F0E0E093ED02F093EE02A091EF02BC
:102E8000B091F002A230E0E0BE0711F00C94A71759
:102E9000A091F102B091F202A430E0E0BE0711F47B
:102EA0000C948A17A830E0E0BE0711F40C948A173E
:102EB000AC30E0E0BE0711F40C948A17A031E0E0DA
:102EC000BE0711F40C948A17A431E0E0BE0711F498
:102ED0000C948A17A831E0E0BE07E1F0AC31E0E0E5
:102EE000BE07C1F0A032E0E0BE07A1F0A432E0E0EE
:102EF000BE0781F0A832E0E0BE0761F0AC32E0E04E
:102F0000BE0741F0A033E0E0BE0721F0A433E0E0CB
:102F1000BE0779F4A091ED02B091EE02A130E0E09D
:102F2000BE0734F4EDE1F0E0E093ED02F093EE0241
:102F30000EC0A091ED02B091EE02A130E0E0BE071C
:102F400034F4ECE1F0E0E093ED02F093EE020E9445
:102F5000020F0E943F31AF9A0E94FD330E9403345A
:102F6000AF988BE18A95F1F70E94EC0264C5E1E528
:102F7000EB1531F5E091EF02F091F0023196E0931C
:102F8000EF02F093F002A091EF02B091F002ECE0BA
:102F9000F0E0EA17FB0734F4E1E0F0E0E093EF0241
:102FA000F093F0020E941334AF9A0E9422340E94E0
:102FB0002834AF988BE18A95F1F70E94EC023BC56B
:102FC000E2E5EB1529F5E091EF02F091F00231977F
:102FD000E093EF02F093F002A091EF02B091F002C3
:102FE000A130E0E0BE0734F4ECE0F0E0E093EF0263
:102FF000F093F0020E941334AF9A0E9422340E9490
:103000002834AF988BE18A95F1F70E94EC0213C542
:10301000E3E5EB1519F5E091F102F091F20231963A
:10302000E093F102F093F202A091F102B091F2026A
:10303000E3E6F0E0EA17FB0734F4E4E0F0E0E093C5
:10304000F102F093F2020E943834AF9A0E944734A2
:103050000E944D34AF980E94EC02EDC4E4E5EB15FC
:1030600011F5E091F102F091F2023197E093F10253
:10307000F093F202A091F102B091F202A430E0E0EC
:10308000BE0734F4E3E6F0E0E093F102F093F202DD
:103090000E943834AF9A0E9447340E944D34AF9852
:1030A0000E94EC02C8C4E5E5EB1581F5E091190337
:1030B000F0911A033097A1F4E1E0F0E0E0931903F6
:1030C000F0931A030E945D34E0E0E0931D03E09367
:1030D0001E03E1E0F0E00E9468340E94733415C0E2
:1030E000E0E0E0931903E0931A030E94252EE0E04C
:1030F000E0931D03E0931E03E0E0F0E00E946834DB
:10310000E0E0ED8BEE8BEF8BE88F95C4E6E5EB15F9
:1031100021F5E0913303F0913403309781F4E1E03D
:10312000F0E0E0933303F0933403ABE3B0E00E94AC
:10313000253AE0E0ED8BEE8BEF8BE88F0DC0E0E001
:10314000E0933303E0933403E0E0F0E0ABE3B0E07E
:103150000E94253A0E9473346EC4E7E6EB1569F4C9
:10316000E1E0F0E0E0931B03F0931C03A3E2B0E086
:103170000E94253A0E94EC025EC4E8E6EB1561F479
:10318000E0E0E0931B03E0931C03E0E0F0E0A3E247
:10319000B0E00E94253A4FC4E9E6EB15E1F4E09176
:1031A0001F03F09120033196E0931F03F093200357
:1031B000A0911F03B0912003E7E1F0E0EA17FB07BD
:1031C0002CF4E0E0E0931F03E09320030E940B3215
:1031D0000E947D3430C4EAE6EB15D1F4E0911F0380
:1031E000F09120033197E0931F03F0932003A09107
:1031F0001F03B0912003109734F4E7E1F0E0E0936F
:103200001F03F09320030E940B320E947D3413C4ED
:10321000EBE6EB15E1F4E0912103F0912203319606
:10322000E0932103F0932203A0912103B0912203A4
:10323000EBE3F0E0EA17FB072CF4E0E0E093210376
:10324000E09322030E9418320E948734F4C3ECE614
:10325000EB15D1F4E0912103F09122033197E09333
:103260002103F0932203A0912103B0912203109730
:1032700034F4EBE3F0E0E0932103F09322030E94A7
:1032800018320E948734D7C3EDE6EB15E9F4E091DC
:103290002303F09124033196E0932303F093240356
:1032A000A0912303B0912403EFE1F0E0EA17FB07BC
:1032B00034F4E1E0F0E0E0932303F09324030E9470
:1032C000E4310E949134B7C3EEE6EB15E1F4E091EE
:1032D0002303F09124033197E0932303F093240315
:1032E000A0912303B0912403A130E0E0BE0734F4A1
:1032F000EFE1F0E0E0932303F09324030E94E43134
:103300000E94913498C3EFE6EB15E9F4E0912503B0
:10331000F09126033196E0932503F0932603A091C4
:103320002503B0912603ECE0F0E0EA17FB0734F444
:10333000E1E0F0E0E0932503F09326030E94F131F1
:103340000E949B3478C3E0E7EB15E1F4E09125039C
:10335000F09126033197E0932503F0932603A09183
:103360002503B0912603A130E0E0BE0734F4ECE081
:10337000F0E0E0932503F09326030E94F1310E94D0
:103380009B3459C3E1E7EB15E9F4E0912703F09191
:1033900028033196E0932703F0932803A091270395
:1033A000B0912803E3E6F0E0EA17FB0734F4E4E029
:1033B000F0E0E0932703F09328030E94FE310E947F
:1033C000A53439C3E2E7EB15E1F4E0912703F0916E
:1033D00028033197E0932703F0932803A091270354
:1033E000B0912803A430E0E0BE0734F4E3E6F0E057
:1033F000E0932703F09328030E94FE310E94A53436
:103400001AC3E3E7EB15E1F4E0912903F0912A03F5
:103410003196E0932903F0932A03A0912903B091F8
:103420002A03E7E1F0E0EA17FB072CF4E0E0E09381
:103430002903E0932A030E944C320E94AF34FBC25E
:10344000E4E7EB15D1F4E0912903F0912A033197D9
:10345000E0932903F0932A03A0912903B0912A0352
:10346000109734F4E7E1F0E0E0932903F0932A03A6
:103470000E944C320E94AF34DEC2E5E7EB15E1F466
:10348000E0912B03F0912C033196E0932B03F09302
:103490002C03A0912B03B0912C03EBE3F0E0EA178F
:1034A000FB072CF4E0E0E0932B03E0932C030E9455
:1034B00059320E94B934BFC2E6E7EB15D1F4E0916E
:1034C0002B03F0912C033197E0932B03F0932C0303
:1034D000A0912B03B0912C03109734F4EBE3F0E0B0
:1034E000E0932B03F0932C030E9459320E94B934CD
:1034F000A2C2E7E7EB15E9F4E0912D03F0912E036A
:103500003196E0932D03F0932E03A0912D03B091FB
:103510002E03EFE1F0E0EA17FB0734F4E1E0F0E01E
:10352000E0932D03F0932E030E9425320E94C334B2
:1035300082C2E9E7EB15E1F4E0912D03F0912E034F
:103540003197E0932D03F0932E03A0912D03B091BA
:103550002E03A130E0E0BE0734F4EFE1F0E0E093A9
:103560002D03F0932E030E9425320E94C33463C2C0
:10357000E1E2EB15E9F4E0912F03F091300331968D
:10358000E0932F03F0933003A0912F03B091300309
:10359000ECE0F0E0EA17FB0734F4E1E0F0E0E09360
:1035A0002F03F09330030E9432320E94CD3443C285
:1035B000E0E4EB15E1F4E0912F03F0913003319753
:1035C000E0932F03F0933003A0912F03B0913003C9
:1035D000A130E0E0BE0734F4ECE0F0E0E0932F032C
:1035E000F09330030E9432320E94CD3424C2E3E2D1
:1035F000EB15E9F4E0913103F09132033196E09359
:103600003103F0933203A0913103B0913203E3E62A
:10361000F0E0EA17FB0734F4E4E0F0E0E093310374
:10362000F09332030E943F320E94D73404C2E1ED8E
:10363000EB15E1F4E0913103F09132033197E0931F
:103640003103F0933203A0913103B0913203A430DF
:10365000E0E0BE0734F4E3E6F0E0E0933103F093FA
:1036600032030E943F320E94D734E5C1EAE2EB15F3
:10367000E9F4E0911303F0911403309759F40E9498
:103680005D34E0E0F0E060E87FE3ED8BFE8B6F8B74
:10369000788F09C00E94252EE0E0ED8BEE8BEF8B3A
:1036A000E88F0E94EC020E94E134C5C1E5E2EB150F
:1036B00011F00C94A91B8BE18A95F1F7E091E902D6
:1036C000F091EA02E0931F03F0932003E091EB02F4
:1036D000F091EC02E0932103F0932203E091ED02DC
:1036E000F091EE02E0932303F0932403E091EF02C4
:1036F000F091F002E0932503F0932603E091F102AC
:10370000F091F202E0932703F0932803E0911F0366
:10371000F0912003A7E2B0E00E94253AE091210356
:10372000F0912203A9E2B0E00E94253AE091230340
:10373000F0912403ABE2B0E00E94253AE09125032A
:10374000F0912603ADE2B0E00E94253A0E94A53434
:1037500072C1EEE5EB1511F00C94FC1B8BE18A9520
:10376000F1F7E0911F03F0912003E0932903F09318
:103770002A03E0912103F0912203E0932B03F093BD
:103780002C03E0912303F0912403E0932D03F093A5
:103790002E03E0912503F0912603E0932F03F0938D
:1037A0003003E0912703F0912803E0933103F09375
:1037B0003203E0912903F0912A03A1E3B0E00E94D3
:1037C000253AE0912B03F0912C03A3E3B0E00E9493
:1037D000253AE0912D03F0912E03A5E3B0E00E947D
:1037E000253AE0912F03F0913003A7E3B0E00E9467
:1037F000253A0E94D7341FC1E4EAEB1531F5949ABB
:10380000959AE0913503F0913603309769F4E1E041
:10381000F0E0ADE3B0E00E94253AE0933503F09389
:1038200036030E94EC020BC0E0E0F0E0ADE3B0E054
:103830000E94253AE0E0E0933503E09336030E94CE
:10384000023394980E94E134F6C0E6EBEB1581F563
:10385000949A959AE0913703F0913803309769F480
:10386000E1E0F0E0AFE3B0E00E94253AE0933703F7
:10387000F09338030E94EC020BC0E0E0F0E0AFE30D
:10388000B0E00E94253AE0E0E0933703E09338038C
:10389000E2E0F0E0E0931703F0931803E1E0F0E0DA
:1038A000E0931103F093120395980E94E134C3C092
:1038B000EAEBEB15A9F4E091CF02F091D0020E945F
:1038C00010390E94983AED8BFE8B6F8B788FE3E86E
:1038D000F1E00E944C3184E00E94DA2D2696ABC0C4
:1038E000EAE5EB1511F00C94E21C0E947D310E9478
:1038F0008A3140F4E8EAF0E0FA93EA9380E00E942B
:10390000DA2D2296E7EFF0E00E944C3184E00E942D
:10391000953140F4E8EAF0E0FA93EA9380E00E94FF
:10392000DA2D2296EEEFF0E00E944C3184E00E9406
:10393000DA2D26960E943F31E5E0F1E00E944C31FD
:1039400084E00E945531ECE0F1E00E944C3184E0CB
:103950000E94643140F4E8EAF0E0FA93EA9380E0F0
:103960000E94DA2D2296E3E1F1E00E944C3184E0DE
:103970000E94D731EAE1F1E00E944C3184E00E94DC
:10398000BB31E1E2F1E00E944C3184E00E94DA2D8B
:103990002696E0910903F0910A030E9410390E94D3
:1039A000983AED8BFE8B6F8B788FE8E2F1E00E9406
:1039B0004C3184E00E94DA2D26960E94EC020E948F
:1039C000192E39C0E2EBEB1571F4E0E0F0E0A5E66A
:1039D000B3E00E94253AE0E0E0936603E0936703DA
:1039E0000E94EC0228C0ECEBEB1569F4E1E0F0E09A
:1039F000A5E6B3E00E94253AE0936603F0936703DF
:103A00000E94EC0218C0EFEDEB15A9F4A7E6B3E0B5
:103A10000E940A3AE130A0E0FA0719F4E0E0F0E091
:103A200002C0E1E0F0E0A7E6B3E00E94253A0E9480
:103A30009F2E0C940000EAE8F1E0BE2E0881699602
:103A40001895F894789460978CE0A4E0B0E0E6E6EE
:103A5000F0E00E94E13B0E94D33B20E030E040E0F8
:103A600050E0F8940E94050534FC08C50E941A0332
:103A70000E94ED34E62DA0913F03B0914003F0E0A9
:103A8000AE17BF072CF4E0E0E093DD02E093DE0226
:103A9000E0E0E0935903E0935A03A0910903B09149
:103AA0000A03A230E0E0BE0751F4A0913F03B091B9
:103AB0004003A230E0E0BE0711F40E94A602E091AC
:103AC0003F03F09140033196A0910903B0910A039E
:103AD000EA17FB0789F4E0E0E0934C03E0934D0321
:103AE000E0934E03E0934F03E0935003E0935103C0
:103AF000E0935203E09353030E94FB3411F00C94C3
:103B0000CF1D0E94F102E0914D03A0914503EA17F9
:103B1000F1F4E0914E03A0914603EA17C1F4E0915D
:103B20004F03A0914703EA1791F4E0915003A0914D
:103B30004803EA1761F4E0915103A0914903EA17A1
:103B400031F4E0915203A0914A03EA1741F1E0E019
:103B5000E0936203E09363030E94063525F821E0B9
:103B600030E041E050E0E1E0F0E0EC8BFD8BEA8BEF
:103B7000FB8BE88BF98BEE87FF87EC87FD87EA8765
:103B8000FB870E94BB010E940C35E093CD02F093AD
:103B9000CE020E94020F0E9417350E94EC02A091F3
:103BA0003B03B0913C03A130E0E0BE0779F4A09163
:103BB0001103B09112030E94BB3B41F4A091170383
:103BC000B0911803AF30E0E0BE070CF013C0E091F5
:103BD000F902F091FA02309739F4E1E0F0E0E09375
:103BE000F902F093FA0205C0E0E0E093F902E093F5
:103BF000FA0205C0E0E0E093F902E093FA02A09136
:103C00000903B0910A03A130E0E0BE0711F00C9463
:103C1000BF1E0E94462E0E942D01E3E00E941D352A
:103C2000662777270E94983AE093FB02F093FC0204
:103C30006093FD027093FE02A091FB02B091FC0222
:103C40008091FD029091FE02EAE0F7ED63E27CE3F1
:103C50000E94243BE093FB02F093FC026093FD0280
:103C60007093FE02A0E0B0E08FE192EC0E94D63AA1
:103C70000E94253510F00C94B31E0E943C3568F468
:103C8000E0E0F0E066E173E4E093FB02F093FC0215
:103C90006093FD027093FE0265C0A091FB02B0919B
:103CA000FC028091FD029091FE020E944B350E9421
:103CB00054350E942D01E5E00E941D35A4E5B3EEC8
:103CC00085E29DE3662777270E94983A0E94243B6D
:103CD000A0E0B0E080E890EC0E94D63A7F936F932A
:103CE000FF93EF93E02FF12FA2EAB7EE8BE396E379
:103CF000662777270E94983A0E94243BDF01CB0178
:103D0000E02FF12F662777270E94983A0E94243BE4
:103D1000AF91BF918F919F910E94F8390E94CF3A45
:103D2000E0935403F0935503609356037093570345
:103D3000E0930303F0930403609305037093060379
:103D4000A0915403B091550380915603909157036D
:103D50000E944B35E093D902F093DA026093DB02C4
:103D60007093DC020CC0E0E0F0E066E173E4E09305
:103D7000FB02F093FC026093FD027093FE020E942E
:103D8000FB3461F583E08A95F1F7772488240E945B
:103D90004E0AA091FF02B09100038091010390911F
:103DA0000203A030E0E0BE07EAEA8E07E2E49E07E5
:103DB00019F00E94C33B91F4E0E0E0936203E093CA
:103DC00063030E94ED340E94BB010E9417350E94DC
:103DD000FB3421F40E944E0A0E94EC02A091FF02E3
:103DE000B09100038091010390910203E0E0F0E0C4
:103DF0006AEF72E40E94973B60F5E0E0F0E060E279
:103E000072EC0E94973B68F4E0E0F0E066E173E456
:103E1000E093FF02F09300036093010370930203A9
:103E200017C0E091CB02F091CC020E941039E093D0
:103E3000D102F093D2026093D3027093D402E09146
:103E4000DD02F091DE023196E093DD02F093DE02B6
:103E50000CC0E0E0F0E066E173E4E093FF02F09371
:103E600000036093010370930203A0910903B091D2
:103E70000A03A230E0E0BE0751F50E946A080E94E2
:103E80002535C8F40E943C3568F4E0E0F0E066E1D6
:103E900073E4E093FB02F093FC026093FD027093E5
:103EA000FE0208C0E091C902F091CA020E941039D6
:103EB0000E9454350CC0E0E0F0E066E173E4E0936A
:103EC000FB02F093FC026093FD027093FE02E89403
:103ED00021F8E89422F8E0916603F09167033097A7
:103EE00031F5A9E0B0E00E94053AA091FF02B0913F
:103EF000000380910103909102030E94973B09F017
:103F000010F40C94851F689421F8ADE0B0E00E9495
:103F1000053AA091FF02B0910003809101039091B6
:103F200002030E94973B10F4689422F825C0A9E090
:103F3000B0E00E94053AA091FB02B091FC02809192
:103F4000FD029091FE020E94973B09F010F40C9440
:103F5000AB1F689421F8ADE0B0E00E94053AA09153
:103F6000FB02B091FC028091FD029091FE020E9442
:103F7000973B10F4689422F8E1E0F0E0E715F805CB
:103F800019F40E9466350EC00E94873539F40E94EC
:103F90006635E1E0F0E07E2E8F2E04C00E942430D2
:103FA000772488240E940C35A091CD02B091CE02D6
:103FB0000E9417390E94CE3B14F40C9490200E946A
:103FC000933511F0689425F825FE89C026FE04C0BB
:103FD0000E940331E89426F827FE04C00E940B31AA
:103FE000E89427F830FE04C00E941331E89430F8BA
:103FF00031FE05C0E0EAF0E00E949E3531F832FE65
:1040000005C0EAEAF0E00E949E3532F8E1E0F0E017
:10401000E417F50721F40E94A63540E050E0E1E006
:10402000F0E0E217F30721F40E94AE3520E030E023
:10403000AC89BD89A130E0E0BE0729F40E94B63505
:10404000E0E0EC8BED8BAA89BB89A130E0E0BE07F4
:1040500029F40E94BE35E0E0EA8BEB8BA889B98990
:10406000A130E0E0BE0729F40E94C635E0E0E88B0D
:10407000E98BAE85BF85A130E0E0BE0729F40E9440
:10408000CE35E0E0EE87EF87AC85BD85A130E0E07E
:10409000BE0729F40E94D635E0E0EC87ED87AA85BB
:1040A000BB85A130E0E0BE0759F4EAEDF0E0E09313
:1040B000F702F093F8020E946E0AE0E0EA87EB87CD
:1040C0000E94933551F00E94DE35E0913F03F0915C
:1040D0004003E0933D03F0933E03E89425F8E0911C
:1040E0001303F0911403309749F4E0913B03F091EE
:1040F0003C03309711F40E946E0A02C00E94C33044
:104100000E940C35A091CD02B091CE020E941739C9
:104110000E94F8390E94D338E093CD02F093CE028A
:10412000A0911903B0911A03A130E0E0BE0711F08D
:104130000C94E520E0911D03F0911E03309711F0DF
:104140000C94E520E0911F03F0912003A091E90277
:10415000B091EA02EA17FB07C1F5E0912103F09163
:104160002203A091EB02B091EC02EA17FB0769F57C
:10417000E0912303F0912403A091ED02B091EE02AF
:10418000EA17FB0711F5E0912503F0912603A091B2
:10419000EF02B091F002EA17FB07B9F4E0912703B0
:1041A000F0912803A091F102B091F202EA17FB0707
:1041B00061F40E94D501E0913303F091340330970C
:1041C00011F40E94150F0E94EC02A0911B03B09104
:1041D0001C03A130E0E0BE0711F00C943421A09143
:1041E0001D03B0911E03A130E0E0BE07E9F5E091A8
:1041F0002903F0912A03A091E902B091EA02EA179B
:10420000FB0791F5E0912B03F0912C03A091EB02B9
:10421000B091EC02EA17FB0739F5E0912D03F0911C
:104220002E03A091ED02B091EE02EA17FB07E1F434
:10423000E0912F03F0913003A091EF02B091F002D2
:10424000EA17FB0789F4E0913103F0913203A09162
:10425000F102B091F202EA17FB0731F40E94EC027E
:104260000E94E6350E945D34A0911503B0911603BB
:104270000E94BB3B4CF4E0911503F09116033F976D
:10428000E0931503F0931603A0911703B091180360
:104290000E94BB3B4CF4E0911703F09118033F9749
:1042A000E0931703F0931803A0911703B09118033C
:1042B000A130E0E0BE07BCF40E94F23514F468942B
:1042C00023F8E0E0E0931103E093120377248824BD
:1042D0000E94873521F4E1E0F0E07E2E8F2E0E94CF
:1042E000FB35949A959AA0910703B0910803A43BDB
:1042F000E0E0BE074CF4E0910703F09108033F961D
:10430000E0930703F09308030E94F23524F46894C5
:1043100023F80E94E134A0916403B0916503A130B9
:10432000E0E0BE0749F4E091CD02F091CE02319673
:10433000E093CD02F093CE02E0910903F0910A03DD
:1043400031970E940736ACF4A5E6B3E00E940A3A22
:10435000309779F4A091FF02B0910003809101039E
:1043600090910203E0E0F0E06BE073E40E94973B81
:1043700000F1E0910903F0910A0332970E94073699
:10438000BCF4A5E6B3E00E940A3AE130A0E0FA07E7
:1043900079F4A091FB02B091FC028091FD02909112
:1043A000FE02E0E0F0E06BE073E40E94973B08F06F
:1043B00064C0A5E6B3E00E940A3AE130A0E0FA0743
:1043C000B1F578868986E091F302F091F40260916C
:1043D000F5027091F602DE0116960E94653AED93A1
:1043E000FC93E091FB02F091FC026091FD02709160
:1043F000FE02E093F302F093F4026093F5027093EF
:10440000F602E1E0F0E07E2E8F2E0E94E134788407
:104410008984EE81FF810E9410390E94983AE093CE
:10442000F302F093F4026093F5027093F60221FE1A
:1044300008C0A0913503B0913603A130E0E0BE077B
:1044400009F003C094980E94990222FE08C0A0912E
:104450003703B0913803A130E0E0BE0709F003C094
:1044600095980E949902A5E6B3E00E940A3AE130CD
:10447000A0E0FA0711F40E94FB3532C0E09141033D
:10448000F09142033196E0934103F0934203A091EF
:104490004103B0914203A230E0E0BE0709F5E0E03D
:1044A000E093E102E093E202E093E302E093E402AE
:1044B0000E94462E0E94FB0EE0913F03F0914003C4
:1044C000E0933D03F0933E030E94DE350E94462EAA
:1044D000E89425F80E94C330E89434F80E9429310A
:1044E0000E940C36E0913D03F0913E030E94073696
:1044F00029F0E0E0E093DD02E093DE02662019F0AF
:104500000E94BB01C39AE0914303F09144033196AA
:10451000E0934303F09344030E94E70378940E94DE
:10452000DA3B669608950E941636E1E0F0E0E093EB
:104530006403F09365030E94231DA0916203B09170
:104540006303A837E0E0BE07B4F4ECE4FDE1FA93BE
:10455000EA930E94A737E0916203F09163033196DA
:10456000E0936203F0936303E0E0E0936403E0937D
:1045700065030E94231D0E94243618950E9416365A
:104580001A930A9300E010E034FCF8C0E0E0E093F6
:104590006203E0936303E89423F8A0911703B091BA
:1045A0001803A431E0E0BE0731F0EAE0F0E0E09368
:1045B0001703F09318030E943236839BDDC0839B60
:1045C0002CC00E943E360F5F1F4FB29B25C021FCBE
:1045D00002C022FE14C0A1E1B0E00E940A3AA0E1AC
:1045E000BEE00E944639E0931503F09316030530B0
:1045F000E0E01E0724F40E94EC0205E010E0EDE28A
:10460000F0E0E017F10741F4E2E0F0E0A7E6B3E004
:104610000E94253A0C940000D2CF0431E0E01E073E
:1046200014F00C94BC23A091F902B091FA02A130CD
:10463000E0E0BE0719F40E9444369EC083999CC0F6
:10464000E89423F8A0911103B09112030E94BB3BA0
:1046500014F40E94EC02A0911103B0911203A13056
:10466000E0E0BE0741F50E944C360E945536E0E07E
:10467000F0E060E371EC0E94973B09F010F40C94B9
:104680004A23ADE0B0E00E94053AADECBCEC8CEC06
:104690009DE308C0ADE0B0E00E94053AA0E0B0E0C4
:1046A00080E89FE30E94D63A0E946636689425F817
:1046B0000E947D3327F8A0911103B0911203A2301C
:1046C000E0E0BE0771F50E944C360E947E36A9E0FC
:1046D000B0E00E94053ADF01CB01E0E0F0E060E3EA
:1046E00071EC0E94973B09F010F40C948023A9E030
:1046F000B0E00E94053AADECBCEC8CEC9DE308C048
:10470000A9E0B0E00E94053AA0E0B0E080E89FE3B5
:104710000E94D63A0E948936689425F80E941B337D
:1047200026F8A0911103B0911203A330E0E0BE0778
:1047300021F40E94A9330E949536A0911103B091F3
:104740001203A430E0E0BE07B9F4A0911303B091C6
:104750001403A130E0E0BE0759F40E94252E0E9408
:1047600095360E94FB0E0E941B31E89425F804C088
:104770000E945D340E9495360E94E7032CC20E947D
:1047800016361A930A9300E010E034FC24C2E0E0ED
:10479000E0936203E0936303E89423F8A091170386
:1047A000B0911803A431E0E0BE0731F0EAE0F0E098
:1047B000E0931703F09318030E943236B29B09C2AC
:1047C000B29B86C00E943E360F5F1F4FE4E1F0E0CF
:1047D000E017F10711F00C9467240E94EC02E0E06E
:1047E000E093F902E093FA02E89423F8949A959AF8
:1047F000E62DEF5FA0910903B0910A03F0E0EA17FC
:10480000FB0769F4E1E0F0E07E2E8F2EE091FB02E1
:10481000F091FC026091FD027091FE020AC07724C3
:104820008824E091FF02F0910003609101037091F0
:104830000203E093F302F093F4026093F5027093A5
:10484000F602E0911103F0911203309751F4E2E087
:10485000F0E0E0931103F093120394980E949536D0
:1048600036C0A0911103B0911203A130E0E0BE0761
:1048700049F4E4E0F0E0E0931103F09312030E94A6
:10488000953625C0A0911103B0911203A230E0E04B
:10489000BE0751F4E1E0F0E0E0931103F09312035E
:1048A00095980E94953613C0A0911103B091120300
:1048B000A330E0E0BE0759F0A430E0E0BE0739F4D1
:1048C000E0E0E0931103E09312030E94E13478CF1B
:1048D0000431E0E01E0714F00C94E925A091F902E0
:1048E000B091FA02A130E0E0BE0719F40E9444360C
:1048F00070C10E94EC02E89423F8B2996AC1E09179
:104900001103F0911203309711F00C945325072CEA
:10491000082879F5A0910903B0910A03A130E0E0DD
:10492000BE07B1F4E3E0F0E07E2E8F2E0E949D36AC
:10493000E0910303F0910403609105037091060375
:10494000E093F302F093F4026093F5027093F602A1
:10495000A0910903B0910A03A230E0E0BE0711F470
:104960000E94A936EAEAF0E0E0930703F093080317
:104970009AC0E1E0F0E0E715F80511F00C9421256C
:10498000A0910903B0910A03A130E0E0BE07A9F5A8
:104990006620E9F4E3E0F0E07E2E8F2EE0E0E09385
:1049A000F902E093FA020E949D36689435F8E0918E
:1049B0000303F09104036091050370910603E093F3
:1049C000F302F093F4026093F5027093F602E1E0D3
:1049D000E61599F40E94AE3635F8E091FF02F091A9
:1049E00000036091010370910203E093F302F093DE
:1049F000F4026093F5027093F602A0910903B0915E
:104A00000A03A230E0E0BE07D9F4E1E0E61511F4B4
:104A10000E94A936E2E0E61599F40E94AE3635F818
:104A2000E091FF02F0910003609101037091020395
:104A3000E093F302F093F4026093F5027093F602B0
:104A400032C0E2E0F0E0E715F80521F50E94C33638
:104A5000E0E0E093F902E093FA02E091FB02F091CA
:104A6000FC026091FD027091FE020E94F3390E94E7
:104A70006F05E091FB02F091FC026091FD027091E4
:104A8000FE02E093F302F093F4026093F502709358
:104A9000F60209C0E3E0F0E0E715F80521F40E9412
:104AA000C3360E949536A0911103B0911203A13034
:104AB000E0E0BE0771F50E944C360E945536E0E0FA
:104AC000F0E060E271EC0E94973B09F010F40C9466
:104AD0007425ADE0B0E00E94053ADF01CB01EDECBA
:104AE000FCEC6CEC7DE30AC0ADE0B0E00E94053A5E
:104AF000DF01CB01E0E0F0E060E87FE30E94F839FD
:104B00000E94CF3A0E946636689425F80E947D3351
:104B100027F8A0911103B0911203A230E0E0BE0784
:104B2000D1F40E944C360E947E360E94E83209F091
:104B300010F40C949E250E94233302C00E942E3351
:104B40000E94F8390E94CF3A0E948936689425F86D
:104B50000E941B3326F8A0911103B0911203A330D9
:104B6000E0E0BE07B9F4EAE0F0E0E0931703F09369
:104B70001803A3E1B0E00E94053ADF01CB01E1E0B8
:104B8000F0E060E070E00E94C93B24F40E9494339E
:104B90000E949536A0911103B0911203A430E0E079
:104BA000BE07B9F4A0911303B0911403A130E0E063
:104BB000BE0759F40E94252E0E9495360E94FB0ED6
:104BC0000E941B31E89425F804C00E945D340E94C5
:104BD00095360E94E703099119910E942436189591
:104BE0006897E0E0EBBBEFEFEABBE0E0E8BBEBEBA4
:104BF000E7BBE0E0E5BBEFEEE4BBE0E0E2BBE2EF09
:104C0000E1BBE0E0E3BFE2BFECBFEFBDEEBDEDBD59
:104C1000ECBDEBBDEABDE9BDE8BDE2BDE5BDE4BD6F
:104C2000E3BDEBB7E06EEBBFE4E0E5BFE0E4E4BF7B
:104C3000E0EEEABFE0E4E9BFE0E8E8B9E0E0E0BFC9
:104C40000E946B02A7E6B3E00E940A3ADF01E1E0AE
:104C5000F0E0EA17FB0744F4E0E0F0E0A7E6B3E099
:104C60000E94253A0E94EC02A7E6B3E00E940A3AAD
:104C7000309729F4E0E00E94C936E9E104C0E2E09F
:104C80000E94C936E8E0E9B90E94D001AE9AA9981D
:104C9000E1E0F0E0E0934303F0934403E0E0F0E070
:104CA00060E070E0E0930D03F0930E0360930F0358
:104CB00070931003EDE2F1E0E093CF02F093D002A5
:104CC000E0E0E0936203E09363030E94E703E1E026
:104CD000F0E0E0930903F0930A03A7E0B0E00E943C
:104CE0000A3AE0930B03F0930C03E1E0F0E0E09369
:104CF0000B03F0930C030E940505A091F102B09103
:104D0000F202A430E0E0BE0714F40E94C603A1E45E
:104D1000B0E00E940A3AE0931303F0931403ECE22C
:104D2000F1E0FA93EA930E94A737E2E0F0E07E2EEA
:104D30008F2EA99A0E949536E0E0E0933B03E09322
:104D40003C03A5E6B3E00E940A3ADF01E2E0F0E0AE
:104D5000EA17FB0734F4E0E0F0E0A5E6B3E00E94D8
:104D6000253AA5E6B3E00E940A3AE0936603F09381
:104D70006703E0E0E093BD02E093BE02E0E0E09371
:104D8000BF02E093C0020E946F0283E08A95F1F7B0
:104D9000AE980E940C300091BF020A930E94F92D38
:104DA0000091BD020E9412301E2F0E944F2E2E2F06
:104DB00083E08A95F1F7AE9A30E040E00E9415302A
:104DC0003D3FEFE74E078CF50E94730283E08A9522
:104DD000F1F7AE980E940C300091BF020A930E9436
:104DE000F92D0091BD020E9412301E2F0E944F2EFD
:104DF0002E2F83E08A95F1F7AE9A30E040E00E94D2
:104E00001530A091BF02B091C002AF37E0E0BE07FD
:104E100059F40E94E83044F4E1E0F0E0E0933B0311
:104E2000F0933C033EEF4FE7CBCF83E08A95F1F759
:104E30000E946B02A1E2B0E00E940A3AE0931903DB
:104E4000F0931A03A3E2B0E00E940A3AE0931B0336
:104E5000F0931C03A5E2B0E00E940A3AE0931D0320
:104E6000F0931E03A7E2B0E00E940A3AE0931F030A
:104E7000F0932003A9E2B0E00E940A3AE0932103F4
:104E8000F0932203ABE2B0E00E940A3AE0932303DE
:104E9000F0932403ADE2B0E00E940A3AE0932503C8
:104EA000F0932603AFE2B0E00E940A3AE0932703B2
:104EB000F0932803A1E3B0E00E940A3AE0932903AB
:104EC000F0932A03A3E3B0E00E940A3AE0932B0395
:104ED000F0932C03A5E3B0E00E940A3AE0932D037F
:104EE000F0932E03A7E3B0E00E940A3AE0932F0369
:104EF000F0933003A9E3B0E00E940A3AE093310353
:104F0000F0933203ABE3B0E00E940A3AE09333033C
:104F1000F0933403A1E4B0E00E940A3AE093130353
:104F2000F0931403AFE3B0E00E940A3AE093370332
:104F3000F0933803ADE3B0E00E940A3AE093350302
:104F4000F0933603A7E1B0E00E940A3AE0933903F8
:104F5000F0933A03ADE0B0E00E94053AE093B90265
:104F6000F093BA026093BB027093BC020E94E70800
:104F70000E94462E0E94E60EE89424F80E94130137
:104F80000E940C36A0910903B0910A03A230E0E020
:104F9000BE0711F00C945928E1E0E61511F00C94CD
:104FA00031280E94D136E093A902ABE1B0E00E9423
:104FB0000E3AE093AA02ACE1B0E00E940E3AE09310
:104FC000AB02ADE1B0E00E940E3AE093AC02AEE17C
:104FD000B0E00E940E3AE093AD02AFE1B0E00E9473
:104FE0000E3AE093AE02A0E2B0E00E940E3AE093E7
:104FF000AF020E949F2EE091A802E03091F5E0916F
:105000006002A9E1B0E00E942D3AE0916102AAE1BC
:10501000B0E00E942D3AE0916202ABE1B0E00E9464
:105020002D3AE0916302ACE1B0E00E942D3AE091AC
:105030006402ADE1B0E00E942D3AE0916502AEE17C
:10504000B0E00E942D3AE0916602AFE1B0E00E942C
:105050002D3AE0916702A0E2B0E00E942D3A0E9452
:105060009F2E0E94D136E093A902ABE1B0E00E94EE
:105070000E3AE093AA02ACE1B0E00E940E3AE0934F
:10508000AB02ADE1B0E00E940E3AE093AC02AEE1BB
:10509000B0E00E940E3AE093AD02AFE1B0E00E94B2
:1050A0000E3AE093AE02A0E2B0E00E940E3AE09326
:1050B000AF02E62DF0E0E0933D03F0933E03E62DD2
:1050C000F0E0E0933F03F0934003689425F8E2EDAD
:1050D000F0E00E949E3525F8A0911903B0911A03C3
:1050E000A130E0E0BE0749F0A0911B03B0911C0382
:1050F000A130E0E0BE0709F023C1A0911D03B091EB
:105100001E030E94BB3B39F4A0911303B09114031A
:105110000E94BB3B09F008C0E0E0E0931303E0937A
:105120001403E0E0F0E006C0E1E0F0E0E0931303F8
:10513000F0931403A1E4B0E00E94253A0E94050513
:10514000A091F102B091F202E0E1F7E20E9446394B
:10515000FF93EF93A091EF02B091F002E4E6F0E04C
:105160000E944639AF91BF91EA0FFB1FA091ED025B
:10517000B091EE02EA0FFB1F0E941039EC8BFD8B01
:105180006E8B7F8B0E94FE2E0E941039E88BF98B6C
:105190006A8B7B8B0E946632FF93EF930E946F3283
:1051A000AF91BF910E947832EC87FD876E877F8731
:1051B0000E948332E887F9876A877B870E9494324E
:1051C000FF93EF930E949D32AF91BF910E94A63250
:1051D000EC83FD836E837F830E94B132E883F98381
:1051E0006A837B830E94DC3614F00C9442290E946F
:1051F000E736F4F4A0911903B0911A03A130E0E06E
:10520000BE07A9F4A0913303B09134030E94BB3BC5
:1052100039F4A0911D03B0911E030E94BB3B09F01D
:1052200002C00E94150F0E94D5010E94EC0229C005
:105230000E94E73621F50E94F236F4F4A09119039A
:10524000B0911A03A130E0E0BE07A9F4A0913303A6
:10525000B09134030E94BB3B39F4A0911D03B0917F
:105260001E030E94BB3B09F002C00E94150F0E9462
:10527000D5010E94EC0202C00E94E63502C00E94E5
:10528000E6355EC00E94DC3611F00C94A029E88956
:10529000F9896A897B89A885B9858A859B850E9459
:1052A000CE3B24F00E94C93B09F04AC00E94E73679
:1052B000F4F4A0911903B0911A03A130E0E0BE0705
:1052C000A9F4A0913303B09134030E94BB3B39F49D
:1052D000A0911D03B0911E030E94BB3B09F002C0C8
:1052E0000E94150F0E94D5010E94EC0229C00E9465
:1052F000E73621F50E94F236F4F4A0911903B0913B
:105300001A03A130E0E0BE07A9F4A0913303B091E5
:1053100034030E94BB3B39F4A0911D03B0911E03DE
:105320000E94BB3B09F002C00E94150F0E94D501EC
:105330000E94EC0202C00E94E63502C00E94E635DF
:10534000662011F00E94BB01E4E1F5E0FA93EA93D4
:105350000E94A7370E94E703A3E4B0E00E940A3A44
:10536000CE2EDF2EE0E0E0935903E0935A03E2E013
:10537000E61511F40E94A602E0910903F0910A03D8
:105380000E940736E1F40E94F1020E941A030E9473
:10539000063525F80E94A6350E94AE350E94B63526
:1053A0000E94BE350E94C6350E94CE350E94D63579
:1053B000EAEDF0E00E949E3525F80E94EC020E9482
:1053C000C7016620D9F044244614C0F45524E8E00F
:1053D0005E1690F4E42DA0E6B2E0F0E0BF93AF9348
:1053E000A9E0B0E00E941E39AF91BF91AE0FBF1F80
:1053F0000E94B72F5394EBCF4394E6CFEEE40E9484
:105400001F2EE6E00E941F2EE7E00E941F2EEFE70E
:105410000E941F2E0E948838E0E0E093F902E0939A
:10542000FA02789423FE09C0AF98C39AAE9AC19845
:105430008BE18A95F1F70E948C38F4CF6896FFCF04
:105440005D9BFECFE881ECB921960895A881B981D2
:105450000E94E339309751F00E94E3393196ED9381
:10546000FC933197DF01EA81EC9304C0EA81EA936F
:105470000E94202A2396089524971A930A93A885B8
:10548000E5E0EA1708F4E887A2E7B0E0E885F0E095
:10549000EE0FFF1FEE0FFF1FEA0FFB1F0E94ED39FB
:1054A000A985BA858B859C850E94D63AE987FA87BB
:1054B0006B877C8700E0E0E0F0E060E87FE3EA8370
:1054C000FB836C837D83EA81FB816C817D81A9856F
:1054D000BA858B859C850E94973B80F0AA81BB8111
:1054E0008C819D81E0E0F0E060E271E40E94243B69
:1054F000EA83FB836C837D830F5FE5CF003029F463
:105500000E94FD36E0E3EC9330C0E02F0150E03024
:1055100061F1AA81BB818C819D810E940437EA835D
:10552000FB836C837D83A985BA858B859C850E94CE
:1055300014370E941A37FF93EF93E12FE05DAF918C
:10554000BF91EC93E12FAA81BB818C819D81FF27C4
:10555000662777270E94983A0E94243BA985BA853E
:105560008B859C850E942137D0CFE885E03019F4E7
:105570000E942A3732C00E94FD36EEE2EC93E885A5
:10558000E150E887EF5F39F1A985BA858B859C8565
:10559000E0E0F0E060E271E40E94243BE987FA87F2
:1055A0006B877C870E94653A1E2F0E941A37FF93F3
:1055B000EF93E12FE05DAF91BF91EC93E12FA985CF
:1055C000BA858B859C85FF27662777270E94983AA6
:1055D0000E942137D4CF0E942A37198108812D9645
:1055E000089524970E94D63BE0E0F0E060E87FE376
:1055F000EB83FC836D837E83AA85E5E0EA1708F4DC
:10560000EA870A85E02F0150E03019F00E942F3719
:10561000F9CFEB85FC856D857E850E94B73B21F433
:1056200020E00E942F373AC02A850E943E3709F0B9
:1056300010F40C94252B0E942F370E943E3720F047
:105640000E9449372F5FF9CF15C00E943E3780F482
:10565000AB85BC858D859E85E0E0F0E060E271E47D
:105660000E94243BEB87FC876D877E872150EDCF1E
:105670000E942F37EB85FC856D857E85A0E0B0E02C
:1056800080E09FE30E94D63AEB87FC876D877E8798
:105690000E943E3718F00E9449372F5F00E0EA85EC
:1056A000E017D0F1AB81BC818D819E810E940437CF
:1056B000EB83FC836D837E83AB85BC858D859E8566
:1056C0000E9414370E945837FF93EF93E12FE05D5B
:1056D000AF91BF91EC93E12FFF27662777270E94B8
:1056E000983AAB81BC818D819E810E94243BAB8521
:1056F000BC858D859E850E94F8390E94CF3AEB8744
:10570000FC876D877E87E02F0F5FE03041F60E94B7
:105710005F37EEE2EC93C3CF0E945F37E985EC93ED
:1057200020302CF40E945F37EDE2EC932195E9E004
:10573000E21764F40E945837FF93EF93A22FEAE038
:105740000E945E39E05DAF91BF91EC930E945837A3
:10575000FF93EF93A22FEAE00E94A639E05DAF919C
:10576000BF91EC93AF81B885E0E0EC930E94DD3B04
:105770002F9608951B7FE989EA93EBA1FCA1FA9388
:10578000EA9364DE403009F04A9508956C970E94D0
:10579000D33B00E0EEA1FFA13196EEA3FFA331972A
:1057A000E4913E2FE03011F40C94D62DE02FE03040
:1057B00039F4353211F401E002C00E946637F5C1B8
:1057C000E130C9F4353221F40E94663700E0EDC1C2
:1057D00002E0E0E0E98B10E03D3211F411E0E5C1B8
:1057E0003B3219F4EBE2E98BE0C1303219F4E0E22C
:1057F000E98BDBC102C0E23039F440E003E0303332
:1058000011F41068D2C102C0E330A1F4303310F0BB
:105810003A3308F009C0A42FEAE0EA9FE02D4E2FAA
:10582000E32FE0534E0FC1C150E03E3211F404E0CB
:10583000BCC111C0E430A9F4303310F03A3308F0A1
:105840000AC01062A52FEAE0EA9FE02D5E2FE32F49
:10585000E0535E0FAAC13C3619F4126005E0A5C101
:1058600004C0E53011F00C94D52DE32FE33631F46C
:105870000E946D37EC910E94743796C1E53411F0A7
:10588000E53609F404C0E63611F00C94892CFE01CB
:105890007296EE83FF830E946D370E94E739E88796
:1058A000F9876A877B87DF01CB010E94BF3B24F029
:1058B000A989AB3249F012C0E885F9856A857B85F4
:1058C0000E943C3A0E947B3717FF04C0E9890E947E
:1058D000743704C00E94FD36E989EC9315FF55E04A
:1058E000363649F40E948237EB85FC85FA93EA93B9
:1058F0000E943C2A09C00E9482373A93EC85FD85BC
:10590000FA93EA930E94F12AFE0172960E948A3766
:105910001EC0E33739F40E946D370E94E7390E94B8
:105920008A370EC0E037C1F40E946D370E94E73914
:10593000EE83FF83FA93EA930E949C370E2F186040
:105940001F77503011F0501708F001C0052F50E0BC
:10595000E0E0E88B20E07BC0E43611F0E93611F49A
:10596000146002C0E537C1F4EAE0E88B11FF0AC019
:10597000E0E0FAEC6AE97BE3EC87FD876E877F87DE
:105980000AE029C0E0E1F7E260E070E0EC87FD8723
:105990006E877F8705E01FC0E83511F4186004C0EA
:1059A000E83711F00C94D42DE0E1E88B11FF0AC028
:1059B000E0E0F0E060E070E1EC87FD876E877F87D4
:1059C00008E009C0E0E0F0E160E070E0EC87FD870E
:1059D0006E877F8704E0503011F01F7701C051E0DF
:1059E00011FF09C00E946D370E94E739E887F987E7
:1059F0006A877B8713C012FF07C00E946D370E9421
:105A0000E3390E94103906C00E946D370E94E339C5
:105A100066277727E887F9876A877B8712FF16C092
:105A2000A885B9858A859B850E94BF3B44F4E8859B
:105A3000F9856A857B850E94E1380E947B37E98978
:105A4000E03019F00F5F5F5F01C01B7F252F10FD55
:105A500014C0041710F4241708F00FC017FF08C073
:105A600012FF04C01B7F3989015001C030E301C01F
:105A700030E20E9466374150ECCF051778F4106190
:105A800012FF04C00E94BA2B01505150E0E30E9463
:105A90007437403009F041505150EFCF202FE88942
:105AA000E030D1F42030B9F013FF04C00E941A375F
:105AB000E49105C0AE81BF81ED91AE83BF83EA93CF
:105AC000EBA1FCA1FA93EA930E94262A403009F048
:105AD00041502150E7CF5FC0EC85FD856E857F8505
:105AE000A885B9858A859B850E947B393E2FE9E090
:105AF000E31730F413FF02C0395C01C0395A01C00A
:105B0000305D14FD22C0E0E3E31760F0AC85BD8595
:105B10008E859F85A130E0E0BE07E0E08E07E0E0E3
:105B20009E0709F40DC0521710F030E309C0421768
:105B300010F010FF01C00EC030E217FF06C030E3C6
:105B4000106112FF02C00E94BA2B0E9466374030DB
:105B500009F041502150EC85FD856E857F85A88533
:105B6000B9858A859B850E94B239E887F9876A875B
:105B70007B87E889AC85BD858E859F85FF27662755
:105B800077270E947B39EC87FD876E877F870E948D
:105B9000B73B09F0A1CF10FF07C0403029F04150BA
:105BA000E0E20E947437F9CF00E0F4CD0E94DA3BC6
:105BB000A8960895F82E22971A930A93DE010E9460
:105BC000CA380A2F1B2FE0E0EA83EB83DE0114962C
:105BD0000E94CA380E94E339FA93EA931A930A930F
:105BE000FE013696FA93EA93D1DD19810881249655
:105BF0000895E881EFB9779BFECFEFB12196089524
:105C00000E9406010E940B010C94110183E48A9505
:105C1000F1F783E48A95F1F70E940F0183E48A95F6
:105C2000F1F708950E940F0183E48A95F1F70C942F
:105C30001101E4E6F0E0FA93EA930C94A737EA93B3
:105C40000E940E38E09361030895E0E0E0931303AF
:105C5000E0931403E0E0F0E0A1E4B0E00E94253A14
:105C60000895E0915903F0915A03A9E0B0E00E9431
:105C70001E39E05AFD4F0895EDB9E0E0EEB9089500
:105C8000E4EFF1E0FA93EA930C94A737EAE0F0E04E
:105C9000FA93EA930C94A737E0E8EA93AACFE0E0FE
:105CA000EA93A7CFE4E0EA93A4CFE1E0EA93A1CF9F
:105CB000EA930E94B3370E2F08958BE18A95F1F78E
:105CC000E7E8EA9396CFE5E1EA9393CFE0E3EA933E
:105CD00090CFE5E4EA938DCF8BE18A95F1F7E8E880
:105CE000EA9387DFD9CF8BE18A95F1F7E9E8EA9368
:105CF00080DFD2CF8BE18A95F1F7EAE8EA9379DF8A
:105D0000CBCFEA9376DFC8CFE02FFF276627772730
:105D10000E94983AE983FA836B837C838BE18A95AE
:105D2000F1F7BDCFE02FFF27662777270E94983A2B
:105D3000E983FA836B837C83E02FF0E00895E1E050
:105D4000F0E0FA93EA930C94A737EFE0F0E0FA93CF
:105D5000EA930E945705E0E1F0E0FA93EA930C948D
:105D60005705ECE2F0E0FA93EA930C945705ECE364
:105D7000F0E0FA93EA930C945705EE87FF87688B5F
:105D8000798BA0913903B0913A03A130E0E0BE07CE
:105D90000895AE85BF8588899989E0E0F0E060E1EB
:105DA00071E40E94243BDF01CB01E0E0F0E060EA17
:105DB00070E40E94563BA0E0B0E080E092E40E94D4
:105DC000D63AEE87FF87688B798B0895EE85FF853D
:105DD00068897989AAE0B7ED83E29CE30E94D63A0C
:105DE0000895AE85BF8588899989EAE0F7ED63E279
:105DF0007CE30E94F8390E94CF3A0895A091E9020D
:105E0000B091EA02E4E6F0E00E944639A091EB028C
:105E1000B091EC02EA0FFB1F0895AE85BF8588891B
:105E20009989E1EEFAEF67EC72E40E94973B0895DE
:105E3000A02FB12FEAE0F0E00E9476390E2F1F2F3D
:105E40000895EAE0F0E00E9476394E2F5F2F089522
:105E5000A42FB52FEAE0F0E00E9446390895DF0153
:105E6000E02FF12FEA1BFB0B0895A22FB32FE4E6DE
:105E7000F0E00E944639F3CFEFE3F0E0FA93EA93C3
:105E80000C945705EAE3F0E0FA93EA930C94570573
:105E900062971A930A93E0E0F0E066E175E4E88B1C
:105EA000F98B6A8B7B8BE0913F03F0914003309735
:105EB0000895E02FF12FDE011296EA0FFB1F0895DF
:105EC000EB81FF2766277727EC87FD876E877F8723
:105ED000AC85BD858E859F85E8E00E94EA38EC8719
:105EE000FD876E877F87EA81AC85BD858E859F851E
:105EF000FF27662777270E94CE38EC87FD876E87BD
:105F00007F870895EC85FD856E857F850E94983A90
:105F1000E88BF98B6A8B7B8BA889B9898A899B89E5
:105F2000E0E0F0E060E077E40E94973B0895A88904
:105F3000B9898A899B89E0E0FFEF6FE777E40E94E7
:105F4000F8390E94CF3AE88BF98B6A8B7B8B0895E6
:105F5000A889B9898A899B89E0E0F0E060E871E46A
:105F60000E94563BE88BF98B6A8B7B8B0895E52D5D
:105F7000F0E0AE0FBF1FEC9162CEEFE8EA9339CEAE
:105F8000E091E502F091E6026091E7027091E8028B
:105F9000A091E102B091E2028091E3029091E402CB
:105FA0000E94CE3B0895E091E102F091E2026091FF
:105FB000E3027091E402A0910D03B0910E03809171
:105FC0000F03909110030E94983A0E94D63AED87F1
:105FD000FE876F87788B0895FA93EA93EF85F889A7
:105FE00069897A890E94F339E0910D03F0910E03DB
:105FF00060910F03709110030E94F3390895ED83AF
:10600000FE836F837887AD81BE818F819885E0E0C4
:10601000F0E068EC72E4089583E08A95F1F7E3E03C
:10602000EA93E7CD0A93E5DD3ACEE12FF0E03E2F8B
:106030004F2F432F3327E22FA32FB42FF0E0EA2B6B
:10604000FB2B3E2F4F2F0895E091FF02F0910003AC
:106050006091010370910203E0935403F0935503A0
:106060006093560370935703E091FF02F091000391
:106070006091010370910203E093F302F093F40244
:106080006093F5027093F602089583E08A95F1F724
:10609000E6E0EA93AEDD83E08A95F1F7089583E0C8
:1060A0008A95F1F7E2E0EA93A4CDE0935803EA93EE
:1060B000A0CDA091EF02B091F002E8EEF3E00E94D3
:1060C00046390895A091ED02B091EE02EAE0F0E0C9
:1060D0000E9446390895A0E0B0E080E291E40E9479
:1060E000243B0E94653AE093C902F093CA020895E6
:1060F0000E940E3AF0E0E093C902F093CA020895BC
:10610000E091C902F091CA020E940239E093C102F3
:10611000F093C202E091C902F091CA02FE2FE0E0C2
:10612000E093C302F093C4020E940239E093C302D9
:10613000F093C4020895E091CB02F091CC020E944A
:106140000239E093C502F093C602E091CB02F091D0
:10615000CC02FE2FE0E0E093C702F093C8020E9459
:106160000239E093C702F093C8020895A091C902D2
:10617000B091CA02E0E6F9E0EA1BFB0BE093C9022A
:10618000F093CA020895E0E0E093DD02E093DE02BE
:10619000E0E0E093DF02E093E002E0E0E093D90288
:1061A000E093DA02E093DB02E093DC020895E1E0A1
:1061B000F0E0EE83FF830C947302E0915803EA93BE
:1061C00018CDEA9316DD88EC90E00197F1F7089579
:1061D000A091BD02B091BE02E6EEF0E0EA17FB0727
:1061E0000895E0EAF0E0E093F702F093F8020E94ED
:1061F0006E0A4CCDEAEAF0E0E093F702F093F80281
:106200000E946E0A43CDE4EBF0E0E093F702F093D6
:10621000F8020C946E0AEEEBF0E0E093F702F093D4
:10622000F8020C946E0AE8ECF0E0E093F702F093C9
:10623000F8020C946E0AE62DF0E0E0933D03F09333
:106240003E03E2EDF0E0E093F702F093F8020C94E5
:106250006E0AE091F302F091F4026091F502709100
:10626000F6020E94F3390E946F050C94EC02E2E002
:10627000F0E0E093F902F093FA020C944909E091FE
:10628000ED02F091EE020E9410390E94983AED8BD7
:10629000FE8B6F8B788F0895FA93EA93EF89F88DD0
:1062A000698D7A8D0E94F339089584DC2696E091F9
:1062B000EF02F091F0020E9410390E94983AED8BA3
:1062C000FE8B6F8B788F089575DC2696E091F10236
:1062D000F091F2020E9410390E94983AED8BFE8BE9
:1062E0006F8B788FAD89BE898F89988DE0E0F0E063
:1062F00060E271E40E94973B0895E091E902F09119
:10630000EA020E9410390E94983AED8BFE8B6F8B47
:10631000788F0895AD89BE898F89988DE0E0F0E08F
:1063200060E271E40E94973B089544DC2696E09178
:10633000EB02F091EC020E9410390E94983AED8B2A
:10634000FE8B6F8B788FE6CFE0E0F0E060E171E4E8
:106350000E94243BDF01CB01E0E0F0E060EA70E462
:106360000E94563BA0E0B0E080E092E40E94D63A62
:106370000E94F33908951EDC2696E0910B03F091FC
:106380000C030E9410390E94983AED8BFE8B6F8BA4
:10639000788F0895A1E1B0E00E940A3A0E94103976
:1063A0000E94983AED8BFE8B6F8B788F089502DCFC
:1063B0002696A1E0B0E00E94053A0E94983AED8B43
:1063C000FE8B6F8B788F0895E0912303F091240367
:1063D0000E9410390E94983AED8BFE8B6F8B788F5C
:1063E0000895E0912503F09126030E9410390E9440
:1063F000983AED8BFE8B6F8B788F0895E091270391
:10640000F09128030E9410390E94983AED8BFE8B80
:106410006F8B788F0895E0911F03F09120030E9405
:1064200010390E94983AED8BFE8B6F8B788F089510
:10643000E0912103F09122030E9410390E94983AC2
:10644000ED8BFE8B6F8B788F0895E0912D03F0918B
:106450002E030E9410390E94983AED8BFE8B6F8BB1
:10646000788F0895E0912F03F09130030E94103946
:106470000E94983AED8BFE8B6F8B788F0895E09198
:106480003103F09132030E9410390E94983AED8B4B
:10649000FE8B6F8B788F0895E0912903F0912A038A
:1064A0000E9410390E94983AED8BFE8B6F8B788F8B
:1064B0000895E0912B03F0912C030E9410390E9463
:1064C000983AED8BFE8B6F8B788F0895A091270300
:1064D000B0912803E0E1F7E20E9446390895A091C7
:1064E0002503B0912603E4E6F0E00E9446390895C2
:1064F000EA0FFB1FA0912303B0912403EA0FFB1FB7
:106500000E9410390895A0911F03B0912003E4E682
:10651000F0E00E944639A0912103B0912203EA0FD6
:10652000FB1F0E9410390895A0913103B0913203EE
:10653000E0E1F7E20E9446390895A0912F03B0915F
:106540003003E4E6F0E00E9446390895EA0FFB1FAD
:10655000A0912D03B0912E03EA0FFB1F0E9410396A
:106560000895A0912903B0912A03E4E6F0E00E9487
:106570004639A0912B03B0912C03EA0FFB1F0E9418
:1065800010390895ED85FE856F857889AD81BE81CE
:106590008F8198850E94C93B0895E0911B03F0917B
:1065A0001C030E9410390E94983AED8BFE8B6F8B72
:1065B000788F0895E0E0F0E060E470E4ED8BFE8B0E
:1065C0006F8B788FE0E0E0931B03E0931C0308954A
:1065D000A9E0B0E00E94053ADF01CB01E0E0F0E085
:1065E00060E271EC0E94973B0895A9E0B0E00E9440
:1065F000053ADF01CB01E0E0F0E06AEF72E40E94CF
:10660000973B0895E2E0F0E0E0931703F09318035E
:10661000E0931103F09312030895E091F302F091D7
:10662000F4026091F5027091F6020E94F3390E9423
:106630006F0568940895E4EBF0E0E093F702F093BF
:10664000F80268940895A9E0B0E00E94053ADF01DD
:10665000CB01EDECFCEC6CEC7DE30895A9E0B0E03F
:106660000E94053ADF01CB01E0E0F0E060E87FE363
:106670000895A9E0B0E00E94053ADF01CB01E0E017
:10668000F0E068E472EC0E94973B0895A091B90293
:10669000B091BA028091BB029091BC02E0E0F0E0C0
:1066A00060E271EC0E94973B0895A091B902B0910D
:1066B000BA028091BB029091BC02E0E0F0E068E495
:1066C00072EC0E94973B0895E091B902F091BA02F2
:1066D0006091BB027091BC02ADE0B0E00E941A3A3A
:1066E000E2E0F0E0E0931703F0931803E1E0F0E05C
:1066F000E0931103F09312030895EEEBF0E0E093C2
:10670000F702F093F80268940895A091B902B0914D
:10671000BA028091BB029091BC02E0E0F0E068EC2C
:1067200072E40E94973B0895A3E1B0E00E94053A0D
:10673000E150F04060407040A3E1B0E00E941A3A9E
:106740000895E8ECF0E0E093F702F093F802689423
:106750000895A3E1B0E00E94053AEF5FFF4F6F4F4D
:106760007F4FA3E1B0E00E941A3A089588EC90E0D0
:106770000197F1F7E2E825CDE091E902F091EA0214
:106780000E2F0A930E94BF370E2F0A9332DA88EC3D
:1067900090E00197F1F708950E94020FE091EB025B
:1067A000F091EC020E9410390E94983AED8BFE8B1A
:1067B0006F8B788F089588EC90E00197F1F7E1E80E
:1067C00000CDE091EB02F091EC020E2F0A930E94B3
:1067D000BF370E2F0A930DDA88EC90E00197F1F79E
:1067E0000895E093ED02F093EE02A091EF02B091D4
:1067F000F002A130E0E0BE07089588EC90E0019738
:10680000F1F7E4E8DECCE091ED02F091EE020E2F1C
:106810000A930E94BF370E2F0A93EBD988EC90E0C1
:106820000197F1F708950E94020FE091EF02F091B5
:10683000F0020E9410390E94983AED8BFE8B6F8B0C
:10684000788F089588EC90E00197F1F7E5E8B9CCEE
:10685000E091EF02F091F0020E2F0A930E94BF37F1
:106860000E2F0A93C6D988EC90E00197F1F70895AE
:106870000E94020FE091F102F091F2020E941039A1
:106880000E94983AED8BFE8B6F8B788F089588EC81
:1068900090E00197F1F7E6E894CCE091F102F091F5
:1068A000F2020E2F0A930E94BF370E2F0A93A1D92E
:1068B00088EC90E00197F1F70895E1E0F0E0E093D3
:1068C0001303F0931403A1E4B0E00E94253A089565
:1068D000A1E2B0E00E94253AE0E0F0E0A5E2B0E0FD
:1068E0000E94253A0895E0E0F0E060E87FE3ED8B58
:1068F000FE8B6F8B788F0C94EC02E0911F03F0916C
:106900002003A7E2B0E00E94253A0C94EC02E0914B
:106910002103F0912203A9E2B0E00E94253A0C94F1
:10692000EC02E0912303F0912403ABE2B0E00E947B
:10693000253A0C94EC02E0912503F0912603ADE298
:10694000B0E00E94253A0C94EC02E0912703F0910C
:106950002803AFE2B0E00E94253A0C94EC02E091EB
:106960002903F0912A03A1E3B0E00E94253A0C9498
:10697000EC02E0912B03F0912C03A3E3B0E00E9422
:10698000253A0C94EC02E0912D03F0912E03A5E33F
:10699000B0E00E94253A0C94EC02E0912F03F091B4
:1069A0003003A7E3B0E00E94253A0C94EC02E0919A
:1069B0003103F0913203A9E3B0E00E94253A0C9430
:1069C000EC02E091F302F091F4026091F502709113
:1069D000F6020E94F3390C946F05E0EFEA93E0E6CB
:1069E000F2E0FA93EA930E941838F0E0E0933F0354
:1069F000F09340030895E0910903F0910A03A091F8
:106A00003F03B0914003EA17FB0708950E94390342
:106A10000E94E90168940895A3E1B0E00E94053A5C
:106A2000A4E0B0E080E090E00E944B390895E4E8F3
:106A3000F3E0FA93EA930C94A737EA930E948D014E
:106A40000E2F1F2FE02FF12F0895E093FB02F093FC
:106A5000FC026093FD027093FE02A091FB02B091D4
:106A6000FC028091FD029091FE02E0E0F0E06AEF0E
:106A700072E40E94973B0895A091FB02B091FC0242
:106A80008091FD029091FE02E0E0F0E060E272ECA5
:106A90000E94973B0895E0E0F0E060E871E40E9416
:106AA000243B0E94653A0895E093D502F093D60204
:106AB0006093D7027093D802E091DF02F091E00278
:106AC0003196E093DF02F093E0020895E091FB023B
:106AD000F091FC026091FD027091FE02E09354037C
:106AE000F09355036093560370935703E091FB02B4
:106AF000F091FC026091FD027091FE02E093F302BE
:106B0000F093F4026093F5027093F6020895E09119
:106B10000903F0910A033197A0913F03B09140031C
:106B2000EA17FB070895E0913D03F0913E03A09121
:106B30003F03B0914003EA17FB070895E093F70283
:106B4000F093F8020E946E0AE8940895E3EDF0E0F5
:106B5000E093F702F093F8020C946E0AE4EDF0E093
:106B6000E093F702F093F8020C946E0AE5EDF0E082
:106B7000E093F702F093F8020C946E0AE6EDF0E071
:106B8000E093F702F093F8020C946E0AE7EDF0E060
:106B9000E093F702F093F8020C946E0AE8EDF0E04F
:106BA000E093F702F093F8020C946E0AE9EDF0E03E
:106BB000E093F702F093F8020C946E0AE2EDF0E035
:106BC000E093F702F093F8020C946E0AE0E0E09391
:106BD0001D03E0931E03E0E0F0E0A5E2B0E00E94B8
:106BE000253A0895A0910703B0910803E3EBF0E084
:106BF000EA17FB070895E0915403F0915503609163
:106C00005603709157030E94F3390C946F05A62D1B
:106C1000B0E0EA17FB070895E0EFEA93E0E6F2E060
:106C2000FA93EA930E9418386E2E08950A921A92E7
:106C3000FA926A937A938A939A93AA93BA93EA936D
:106C4000FA93EFB7EA930895E991EFBFF991E991CB
:106C5000B991A9919991899179916991F990199036
:106C600009900895E9EAF0E0E0930703F093080340
:106C7000E2E3F0E0FA93EA930C94A737E2E3F0E062
:106C8000FA93EA930C94A737E0E0E093F902E093DB
:106C9000FA020E94EC0295CEEAE0F0E0E0931703DE
:106CA000F0931803E1E0F0E00895E0933703F093E8
:106CB0003803E1E0F0E0AFE3B0E00E94253AADE058
:106CC000B0E00E94053ADF01CB010895ADE0B0E0ED
:106CD0000E941A3AADE0B0E00E94053AE093B90292
:106CE000F093BA026093BB027093BC02E0E0F0E064
:106CF00060E070E00E94F3390C946F05E093350377
:106D0000F0933603E1E0F0E0ADE3B0E00E94253A15
:106D10000895A9E0B0E00E941A3AE0E0F0E060E0F7
:106D200070E00E94F3390C946F05E0E0F0E060E061
:106D300070E00E94F3390C946F05E0910303F09129
:106D4000040360910503709106030E94F3390C94CB
:106D50006F05E2E0F0E07E2E8F2EE7CF77248824C7
:106D6000E0E0E093F902E093FA02E091FF02F09193
:106D7000000360910103709102030E94F3390E94A5
:106D80006F0568940895E72DF82D31977E2E8F2E8C
:106D90000895EBB9E8E9EAB9E6E8E0BDE0E0E0BD76
:106DA0000895A9E1B0E00E940E3AE093A802AAE19A
:106DB000B0E00E940E3A0895EC89FD896E897F89C2
:106DC000AC85BD858E859F850E94C93B0895EC8961
:106DD000FD896E897F89AC81BD818E819F810E94F2
:106DE000C93B0895E889F9896A897B89A881B981B5
:106DF0008A819B810E94C93B0895AE81BF81119613
:106E0000AE83BF8311970895E0E0F0E060E271E4A3
:106E10000E94563BA0E0B0E080E09FE30E94D63A9B
:106E20000E94F3390C94C1380E94563B0E94653A87
:106E30001E2F0895EE81FF813196EE83FF833197F7
:106E400008950E94F8390E94CF3AE987FA876B8744
:106E50007C870895AE81BF81E0E0EC930895AB811B
:106E6000BC818D819E81E0E0F0E060E271E40E94EF
:106E7000243BEB83FC836D837E830895EB81FC814F
:106E80006D817E81AB85BC858D859E850E94973BFB
:106E90000895AB85BC858D859E85E0E0F0E060E2DD
:106EA00071E40E94563BEB87FC876D877E870895CF
:106EB000EF81F8853196EF83F88731970895AF8198
:106EC000B8851196AF83B887119708953A93EBA1CF
:106ED000FCA1FA93EA930C94262AACA1BDA11497C5
:106EE000ACA3BDA314960895EA93EBA1FCA1FA9379
:106EF000EA930C94262AE887F9876A877B87EDE274
:106F0000E98B0895E885F9856A857B850E94F339C8
:106F10005A930895EE83FF83FA93EA930E9492377F
:106F20000E2F0895A991B991EE27FF276D91662341
:106F300011F03196FBCF0895AA27BB27E991F9916B
:106F40000590002011F01196FBCFFD010895E99105
:106F5000F991309639F080ED97E00197F1F7A89517
:106F60003197C9F70895E881E295EF70AE2FAA0F27
:106F7000AA0FEA0FEE0FA991AF70EA0F0895A99139
:106F8000EE27AA5012F0E05FFCCFA65FEA0F08954B
:106F9000EE27C398BB9A80EC93E00197F1F7BB987A
:106FA00085E28A95F1F7B39B08958BEC8A95F1F70A
:106FB000B39BE3958CE093E00197F1F70895BB9ABA
:106FC00085E08A95F1F7BB988DE18A95F1F7889471
:106FD000B3990894E79585ED8A95F1F70895E894BB
:106FE000BB9A85E08A95F1F770FDBB9883E28A959C
:106FF000F1F7B39903C070FF03C0089570FF0895BF
:1070000088EC8A95F1F7BB988DE08A95F1F7689442
:10701000089568E0D4DF6A95E9F7089568E079910A
:10702000EE27DDDF26F477956A95D9F7E395089585
:107030004F935F9311244427A881B981012C112417
:10704000A7DFEE23F9F0EA81EA93E8DF51E050157B
:1070500098F4B5DFE7FD08C0B2DFE7FD06C03FD01A
:10706000892319F4152E01C0AADF39D0892370E0D5
:1070700009F071E0B4DF1EC0A2DFE7FF0BC09FDFA5
:10708000E7FF05C0E42F5F914F9123960895689420
:1070900037D0EFCF94DFE7FF01C003C0501531F0C8
:1070A000152EE8942DD077279ADF04C0689428D055
:1070B00071E095DF5395513454F281DFEE1FEE1FDE
:1070C000E1701896EC93189743951120D9F259E086
:1070D000EC911996EC9318975A95D1F7AFCFE52F0D
:1070E000EA956E2FE695E695E695FF27EA0FFB1FDA
:1070F000808191E0677019F0990F6A95FCCF08952F
:10710000EEDF1EF09095892301C0892B80830895BE
:10711000E5B7E068E5BF0895E5B7EF78E062E5BF61
:10712000889508957B816A81F981E88177FB770FE3
:1071300067FD7160972F9E5781F078F0983190F439
:10714000AA27BB27882708948795B795A7959A956E
:10715000D1F7EA23FB23682305C0E8947727EE27BD
:10716000FF2766276F77769508F4606877F9A9910D
:10717000B99189919991EA17FB076807790797FBFD
:107180000895D0DF09F40895F6F79FEBAA27BB27EF
:1071900080E80CC20024AF0DB01D0895EA0FFB1F5C
:1071A000681F791F0895EA1BFB0B680B790B089584
:1071B000EA2BFB2B682B792B0895E095F0953196FF
:1071C0000895E095F09560957095EF5FFF4F6F4FD4
:1071D0007F4F0895EE230E2EFD01BC0131F0EE0F1E
:1071E000FF1F661F771F0A94D1F70895EE230E2E16
:1071F000FD01BC0131F075956795F795E7950A9407
:10720000D1F70895EF2FFF27E7FDFFEF0895F0E096
:1072100060E070E0E7FF0895FFEF6FEF7FEF089504
:1072200060E070E0F7FF08956FEF7FEF089580E072
:1072300090E0B7FF08958FEF9FEF0895FA9FF02D2C
:10724000EB9FF00DEA9FE02DF10D08957A9F702DD0
:107250006B9F700DF89F700DE99F700D6A9F602DF8
:10726000710DFB9F600D711DE89F600D711D8827DA
:10727000FA9FF02D610D781FEB9FF00D611D781FB7
:10728000EA9FE02DF10D681F781F08957BD0D6DFAF
:107290000EF493DF089584D0D9DF0EF492DF0895C1
:1072A000002498E0AA0F001C0E1A10F40E0E01C064
:1072B000A1609A95B9F7EA2FA02D089557D0F0DF75
:1072C0000EF4E19508950024112490E1AA0FBB1F4C
:1072D000001C111C0E1A1F0A18F40E0E1F1E01C0EE
:1072E000A1609A9599F7FD01D00108954BD0EBDF8D
:1072F0000EF463DF08953F934F935F9300241124AE
:107300003327442750E2AA0FBB1F881F991F001C78
:10731000111C331F441F0E1A1F0A360B470B28F48B
:107320000E0E1F1E361F471F01C0A1605A9559F748
:10733000FD01BC01D001832F942F5F914F913F91AC
:1073400008952ED0D8DF0EF43CDF0895E894A7FF0F
:1073500002C0A1956894E7FDE195A2DFEA2F0EF443
:10736000E1950895C8DFFD01BC010895E894E7FFA9
:1073700002C0E1956894A7FF04C0A19500F80394AA
:1073800000FA0895E894F7FF02C017DF6894B7FF8A
:1073900006C0A095B095119600F8039400FA0895E0
:1073A000E89477FF02C00DDF689497FF0BC00024BC
:1073B000A095B095809590951196801D901D00F830
:1073C000039400FA0895ED91FC9111970895ED91C1
:1073D000FD916D917C91139708950590159065919D
:1073E0007491F00108957A936A93FA93EA93089559
:1073F000182E862F612D192E972F712D1B2EBF2F22
:10740000F12D1A2EAE2FE12D0895129603D07F2F65
:107410006E2F1297119602D0FE2F1197E199FECF91
:10742000FF93FFB7F894AEBBBFBBE09AEDB3FFBFCD
:10743000FF9108950AD012960E2E1F2EE62FF72FD9
:1074400004D0E02DF12D1297089507D01196EF93F7
:10745000EF2F03D0EF9111970895E199FECF9FB7D9
:10746000F894AEBBBFBBE09A8DB3E81719F0EDBB43
:10747000E29AE19A9FBF089530976040704009F00A
:107480007058089550E8572711F45F93D1C05F3FBB
:1074900031F0660F000C57956795752F08955F932F
:1074A00000200AF0CBC0BEC050E8192E1522880F6C
:1074B000991F9527550F879550E8072E0522660FCF
:1074C000771F7527550F679508955F93F5DF70381F
:1074D00018F07F3F08F4ACC056E1571B92F4519569
:1074E000583028F0EFEFFFEF6FEF7FE71AC07727F4
:1074F0005523B9F0EE0FFF1F661F771F5A95D1F77E
:1075000010C07727583028F0EF2FF62F672F5850EC
:10751000F9CF552331F076956795F795E7955A950C
:10752000D1F700200AF44DDE5F910895689401C000
:10753000E894309760407040B1F0002426F0772343
:1075400012F400943EDE172E7EE1112032F07A957F
:10755000EE0FFF1F661F111CF9CFEF2FF62F612DC5
:107560005F9390DF5F9108955E2FEA2FA52F5F2F25
:10757000FB2FB52F562F682F852F572F792F952F3B
:10758000502D012C152E0895EA0FFB1F681F08953A
:10759000E095F0956095EF5FFF4F6F4F08955F9313
:1075A00083DF903871F150E8152604C05F937CDFCB
:1075B000903839F1703821F1572F591B13F112F41B
:1075C000D3DFFACF583118F0AA27BB2788275830C5
:1075D00028F0AB2FB82F88275850F9CF552329F022
:1075E0008695B795A7955A95D9F7502D512562F0F4
:1075F000CBDF38F46795F795E795739513F41EC0C4
:10760000B3DF40DF5F910895EA1BFB0B680B81F04D
:1076100010F40094BDDF6623A2F3EE0FFF1F661F78
:107620007A95CBF7EFEFFFEF6FE77FEF5F9108956C
:10763000EE27FF27662777275F910895EFEFFFEF8B
:107640006FE77FE75F9108955F932EDF703881F3D6
:10765000903871F301240894791F23F44CF300202F
:107660000AF3ECCF3F934F93112433274427552738
:1076700098E1330F441F551FEE1FFF1F661F30F4A4
:107680003A0F4B1F581FE11DF11D611D9A9589F797
:107690004F913F9166232AF0550FEE1FFF1F661F83
:1076A00002C07395E3F2EEDE5F9108955F93FCDE16
:1076B000703819F4112012F6B5CF903809F4B8CF0C
:1076C00001240894970B1BF4D4F30020F4CF792FF6
:1076D0006695F795E7958695B795A7954F931124ED
:1076E0004427552798E1AE17BF07860728F0AE1B41
:1076F000BF0B860B089401C08894111C441F551FB2
:10770000AA1FBB1F881F9A9571F7E12DF42F652FD3
:10771000A695E91FF91F691F4F9166232AF0EE0F06
:10772000FF1F661F7A955BF2ADDE5F910895992386
:107730009AF0772342F0971748F029F4AE17BF0765
:10774000860720F031F098948894089598940894CE
:1077500008951894889408957723C2F7971798F39B
:10776000A9F7EA17FB07680788F399F3ECCF30977E
:1077700060407040089500240A160B060895109783
:1077800080409040089500240A160B06080609065A
:107790000895EA17FB07680779070895AE17BF0732
:1077A0008607970708955A934A933A932A931A9310
:1077B0000A9308955D814C813B812A81198108815A
:1077C0000895AC0FBD1F05900D928A95E1F70895BD
:00000001FF
